:10000000D6C400000EC500000CC500000AC50000E3
:1000100008C5000006C5000004C5000002C50000B8
:1000200000C50000FEC400000C946E4E0C942952D2
:100030000C94374DF6C40000F4C40000F2C4000074
:10004000F0C40000EEC40000ECC40000EAC40000EC
:10005000E8C400000C947B4DE4C40000E2C400003E
:10006000E0C40000DEC40000DCC40000DAC400000C
:10007000D8C40000D6C40000D4C40000D2C400001C
:100080000C948920CEC40000CCC40000CAC4000077
:10009000C8C40000C6C400002B0014001A000800E9
:1000A000150017001C0018000C00120013002A0095
:1000B000290004001600070009000A000B000D00CB
:1000C0000E000F0033003400E1001D001B0006008D
:1000D00019000500110010003600370038001E7CA2
:1000E0000000E000E200E30021522C002C0022522C
:1000F0005000510052004F0035021E021F02200224
:1001000021022202230224022502260227022A00BB
:100110004C003A003B003C003D003E003F002D02F9
:100120002E022F0230023102010040004100420045
:10013000430044004500320264024A004D000100C1
:100140000100010001000100010001000100235233
:10015000AB00AA00A900AE0035001E001F00200061
:1001600021002200230024002500260027002A0069
:100170004C003A003B003C003D003E003F002D009B
:100180002E002F00300031000100400041004200ED
:10019000430044004500320064004B004E00010063
:1001A00001000100010001002352010001000100D3
:1001B000AB00AA00A900AE000100007C0100010014
:1001C00001000100010001000100010001004C00DC
:1001D0000100010001000100010001000100010017
:1001E0000100010001000100010001000100010007
:1001F00001000100010001000100010001000100F7
:1002000001000100010001000100010001000100E6
:10021000010001000100010000021222000313236B
:1002200000041424000A1A2A000B1B2B000C1C2C9F
:10023000010212220103132301041424010A1A2AC1
:10024000010B1B2B010C1C2C000515250006162686
:1002500000071727000D1D2D000E1E2E000F1F2F4B
:10026000010515250106162601071727010D1D2D6D
:10027000010E1E2E010F1F2F008070600081716122
:10028000008272620088786800897969008A7A6AD7
:1002900001807060018171610182726201887868F9
:1002A00001897969018A7A6A0083736300847464BE
:1002B00000857565008B7B6B008C7C6C008D7D6D83
:1002C000008E7E5D018373630184746401857565AE
:1002D000018B7B6B018C7C6C018D7D6D00010101BC
:1002E00001010101010102020202020202020203F3
:1002F00003030303030303040404040404040505C3
:100300000505050606060606070707070708080885
:1003100008090909090A0A0A0B0B0B0C0C0C0D0D34
:100320000D0E0E0E0F0F0F101011111112121313CC
:100330001414151516161717181819191A1A1B1B45
:100340001C1D1D1E1E1F20202122222324242526A1
:1003500026272829292A2B2C2D2D2E2F30313232D9
:10036000333435363738393A3B3C3D3E3F404142E5
:10037000434445464748494A4C4D4E4F50515354CB
:10038000555658595A5B5D5E5F616264656668697F
:100390006B6C6D6F7072737577787A7B7D7E8082FF
:1003A000838587888A8C8E8F91939596989A9C9E48
:1003B000A0A2A3A5A7A9ABADAFB1B3B5B7BABCBE58
:1003C000C0C2C4C6C9CBCDCFD1D4D6D8DBDDDFE225
:1003D000E4E7E9EBEEF0F3F5F8FAFDFF01000100C8
:1003E00054139E10F21000000200020050139E10E1
:1003F000F21000000300010055139E10F2100000DF
:10040000040002003A139E10F210F80B05000100E0
:1004100056139E10F2100000060002003C139E10BE
:10042000F21000000700020052139E10F2100000AC
:100430001200020058139E10F21000001300020078
:100440005A139E10F2100000140001005C139E105D
:10045000F2100000150000000000010C101B00004D
:10046000160001005713B510091100001700010113
:100470005713B51009110000180001025713B510E9
:1004800009110000190002005E139E10F210000016
:100490001A0001035713B510091100001B000200D8
:1004A00060139E10F2100000FD377A585A000004C5
:1004B000E6D6B4460200210116000000742FE5A321
:1004C000E002BE011C5D003D8889C65436C3174F4B
:1004D000E4E3C86AC77732D0380A4B88486EC893BD
:1004E00063DA057E4FAAA4EB947F6698F2AEB3BFA1
:1004F0000E6976BE4D3EED10C5B090C6A0C427482B
:10050000E34F982A80F13AB8E568D700EED00D3570
:1005100097ED23E197321D1AAA213D958C621B4469
:100520003636A5339152999E0A70A22D4FB7068593
:1005300075E8EC8B6F18159BCB69253B0A7AC78D44
:10054000D7597EF3643F7DB236541B80BE5031BA1A
:100550001CF6D010452E8F29CFBDB7D2CB3CB1C1F0
:100560005DDA6A3A8F288808E31D1C66C8FD4DB421
:10057000F6F0BE74539C6B4910FD56B65A0D3220EE
:100580004788E6227FC67BC44EC549012A054A7AC0
:10059000F42C384B82E3D800CE910E2E4CD9D36088
:1005A000B04C78F45DE31F6317C516A9B47779E002
:1005B0008DA73A941A0AC4EB8FF062F48EE4E1E35B
:1005C00043B8F54ABFC387DBE85548F6A6ACD188E7
:1005D000657D131F62C275EE436612006438129186
:1005E0004D310000B141A0DF9E16198A0001B8020A
:1005F000BF050000828AD60CB1C467FB0200000070
:100600000004595A0000000001002D000200010002
:1006100003000200040003000500040006000500BA
:100620000700060008000700090008000A0009008A
:100630000B000A000C000B000D000C000E000D005A
:100640000F000E0010000F0011001000120011002A
:1006500013001200140013001500140016001500FA
:100660001700160018001700190018001A001900CA
:100670001B001A001C001B001D001F001E00200094
:100680001F0021002000220021002300220024005E
:10069000230025002400260025002700260028002E
:1006A0002700290028002A0029002B002A002C00FE
:1006B0002B001C002C001E004C4C4C4C4C4C2A5265
:1006C000525252524C4C4C4C4C4C2A525252525256
:1006D0004C4C4C4C4C4C2A52525252524C4C4C4C5E
:1006E0004C4C005252525252504F52514A4D4B4E66
:1006F0002A4C2F30B6B7ABACBBBCA9AABDBE0D0E01
:100700000B0F1A0508050905071811130408120C28
:1007100005010980A101850319012AB700150126E9
:10072000B700950175108100C0050C0901A1018574
:100730000419012AA002150126A002950175108155
:1007400000C005010906A1018506050719E029E792
:10075000150025019508750181020507190029EF8B
:100760001500250195F0750181020508190129057B
:10077000950575019102950175039101C00660FF11
:100780000961A1010962150026FF00952075088105
:10079000020963150026FF00952075089102C00527
:1007A000010906A101050719E029E71500250195B2
:1007B0000875018102950175088101050719002955
:1007C000FF150026FF009506750881000508190130
:1007D00029051500250195057501910295017503FF
:1007E0009101C000000000000000000000000000B7
:1007F00000000000000000000000000000000000F9
:10080000000000000000007E0F00D4FFFFFFC700C3
:1008100000007800000000000000002A2B280000E3
:10082000000000000000000000000000000029009F
:100830000000002C1E3420212224342627252E36A9
:100840002D3738271E1F2021222324252633333617
:100850002E37381F0405060708090A0B0C0D0E0F6A
:10086000101112131415161718191A1B1C1D2F31ED
:1008700030232D350405060708090A0B0C0D0E0F51
:10088000101112131415161718191A1B1C1D2F31CD
:1008900030354C0902BF00050100A0FA0904000030
:1008A0000103010100092111010001224400070593
:1008B000810308000109040100020300000009216E
:1008C0001101000122220007058203200001070513
:1008D00003032000010904020001030000000921B4
:1008E00011010001226D0007058403200001080B9F
:1008F00003020101000009040300000101000009D6
:10090000240100010900010409040400020103009C
:100910000007240100014100062402010100062411
:100920000202020009240301030102010009240359
:10093000020401010100090506024000050000054E
:10094000250101010905850240000500000525017A
:1009500001031201000200000008A803A2BE01006A
:10096000010203011C037600690061006C003A007B
:10097000660036003400630032006200330063001A
:1009800000001A0350006C0061006E0063006B00F1
:1009900020004C00690067006800740000000A0332
:1009A0004F004C004B0042000000040309041124D6
:1009B0001FBECFEFD0E2DEBFCDBF04B603FE18C02E
:1009C0008091851390918613A0918713B09188131D
:1009D0008730904BA740B04B59F41092851310927A
:1009E00086131092871310928813E0E0F0EF0995B8
:1009F00023E1A4E9B5E001C01D92A538B207E1F7F3
:100A000015E0A0E0B1E0ECE6F3EC00E00BBF02C0C3
:100A100007900D92A439B107D9F70E94443A0C947B
:100A2000C760EECA9C019A9581159F4118F5F32F76
:100A3000F270EE27832F8170732F74706627532F07
:100A40005870442734FF0CC08295807FEF2B09F04B
:100A50008062672B09F08064452B69F080680895F7
:100A6000EF2B09F08260672B09F08460452B19F0A9
:100A70008860089580E00895CF93DF93EB01D2DF83
:100A8000FE010995DF91CF9108950C94665F08955A
:100A9000982F92959F7024E0911102C020E0982F2A
:100AA000892F86958695811511F02E5F982F892FB5
:100AB0008695820F0895282F92959F70963099F011
:100AC00060F4925F9F70923030F4203FB1F038F4C0
:100AD00081E0283E38F080E008959A5FF3CF81E00E
:100AE000243FC9F7089591E0813F09F090E081E04B
:100AF000283E08F080E0892B089581E008958093D6
:100B00003813089580933913089521E030E001C02F
:100B1000220F8A95EAF780913913822BF3CF21E0D7
:100B200030E0A90102C0440F551F8A95E2F7CA01BF
:100B30008095909139138923E5CF9091391321E065
:100B400030E0F90101C0EE0F8A95EAF7D90102C041
:100B5000AA0FBB1F6A95E2F7EA2B01C0220F4A9544
:100B6000EAF7892F8E23E81303C0892F822BCACF7F
:100B70002095822F8923FBCF8091220C90E020E0EA
:100B8000022E001C0008281709060CF008952F5F9C
:100B9000F7CFFC01DB018481813041F514968C9103
:100BA0001497813019F591818CE0E081F0E0899F04
:100BB000E00DF11D1124E854F94F94919A32B1F0EF
:100BC00011962C911197EC91F0E0829FE00DF11DB0
:100BD0001124E854F94FE49181E09E1301C080E0B4
:100BE00091E0EA3209F090E0892B089581E00895C0
:100BF0009C018091DA118D79811119C0211540E590
:100C0000340780F4211580E23807C0F4233331051E
:100C100011F1D0F481E02E31310590F4243031050A
:100C200030F00895C90196558115914010F080E08B
:100C30000895C901805F96450797C8F33327E6CF2B
:100C40002C323105A1F708952653310981E0233074
:100C5000310538F3ECCF81E0089580918B0C9091B1
:100C60008A0C981301C008958F5F8770FACF909116
:100C7000DE11809589238093DE11282F27702111A2
:100C800010C0891771F09091631392FF0AC0869586
:100C90008695869544DF1092DE111092E011109235
:100CA000DF1108959091DA11982B9093DA1108953D
:100CB000982F90958091DD1189238093DD110895FF
:100CC0008091D811811531F01092D8111092D7115E
:100CD0001092D6110895803E9105D9F1C8F4813360
:100CE000910509F482C048F48932910509F472C073
:100CF0008A32910509F480C0089589339105E9F09D
:100D000082389105D1F08533910509F45EC00895CC
:100D1000843E9105D9F148F4823E910539F1833E34
:100D2000910549F181EE90E00895863E9105C9F163
:100D3000873E910509F43EC0089520916213237007
:100D4000211164C02091631323FF14C089E290E055
:100D500008952091621320FD45C03091631330FF48
:100D600009C024FD24C083EE90E008952091621311
:100D700022FDF7CF08952091621322FD44C03091E7
:100D8000631330FD43C024FFF5CF11C020916313DE
:100D900021FFF0CF8091621384FD09C087EE90E0BF
:100DA00008952091621323FFE5CF24FFF7CF80E061
:100DB00090E008952091621323FD2BC030916313BE
:100DC00031FFE1CF84EE90E008952091621325FF7A
:100DD000D1CFBCCF2091621325FD1EC0209163139B
:100DE00023FFC8CF89E390E008952091621326FF86
:100DF000C1CF8AE290E008952091621326FFBACF16
:100E000081E390E0089582EE90E0089580EE90E016
:100E1000089586EE90E0089585E390E0089590911E
:100E2000621392FF10C041E0282F2471243009F092
:100E300040E031E0282F2871283009F030E04317D6
:100E400011F02CE0822793FF10C041E0282F24717D
:100E5000243109F040E031E0282F2871283109F0D1
:100E600030E0431711F02CE082273091631330FFFC
:100E700010C051E0282F2171213009F050E041E0ED
:100E8000282F2871283009F040E0541711F029E08C
:100E9000822731FF10C041E0282F2171213109F054
:100EA00040E031E0282F2871283109F030E0431765
:100EB00011F029E0822794FD877E08951F93CF9338
:100EC000DF9309DFEC01811522E5920708F052C09B
:100ED000811540E5940708F0CDC0803E910520F5CE
:100EE0008D3C910508F0A1C0883A910570F4853ACF
:100EF000910508F097C081309105B9F10497813AC6
:100F0000910598F1C0E0D0E030C0885A91094B9724
:100F1000C8F7C85AD0E0CC0FDD1FC75EDA4F099082
:100F2000D881C02DD46421C0811550E49507B0F458
:100F3000C11580E2D80708F0B3C0C83ED105A8F0BB
:100F4000CE019A9581159F41E8F68D2F68DF182F05
:100F5000CE019927C0DEEC01D12B07C09927BBDE5B
:100F6000CC27DF70C82BD92BD06ACE01DF91CF916F
:100F70001F910895803842E59407C8F5803652E500
:100F8000950708F05BC0C03482E5D807D0F4C032C2
:100F900092E5D90708F04BC08C2F8695869520E204
:100FA000829FC0011124C37021E030E0A90102C07A
:100FB000440F551FCA95E2F7EA01C82BD92BDD680B
:100FC000D4CF8C2F86958695877050E2859FC0017F
:100FD0001124C37021E030E0A90102C0440F551F65
:100FE000CA95E2F7EA01C82BD92BDC68BECF803C5A
:100FF00052E5950758F48F71C03AD245A0F590E0BC
:10100000982F8827EC01C46FD06AAFCF805C9245DF
:10101000809708F077CFDC2FCC27CC27DF71C06F0B
:10102000D06AA3CFA497D064A0CFD0659ECFCF7154
:10103000D0E0DC2FCC27C16FD06A97CF86958695FC
:10104000877020E2829FC0011124C37021E030E04C
:10105000A90102C0440F551FCA95E2F7EA01C82B47
:10106000D92BDA6882CFDBDEC82FD0E0DC2FCC278B
:10107000D0627BCF8F71D3DE93E0CC0FDD1F9A95CA
:10108000E1F7CC27DF70282F30E084FF05C050E166
:10109000859F900111243327C22BD32BD06965CFB4
:1010A0008D2F8F71BCDE182FCE01992714DEEC0135
:1010B000D12BDECF80E00895EF92FF920F9397013E
:1010C000201B3109211591E0390710F02FEF30E096
:1010D0002095382F320F08F43FEF832F0F91FF90A8
:1010E000EF900895EF92FF920F939701201B310923
:1010F000211541E0340710F02FEF30E0322F30950A
:10110000482F430F08F44FEF842F620F0F91FF9089
:10111000EF900895EF92FF920F93972FFA01B90184
:101120009701093430F4201B3109211541E03407BF
:1011300010F02FEF30E03896719740F0AB01485F28
:101140005F4F4131510510F02FEF30E02095382FDF
:10115000320F08F43FEF832F77FF02C06D5F7F4FA0
:1011600075956795759567952091D00B620F792FCE
:101170000F91FF90EF900895EF92FF920F93E00E82
:10118000F11CF90137FF03C0F195E195F10924E065
:10119000EE0FFF1F2A95E1F7E11531E0F30714F098
:1011A000EFEFF0E09A0157FF03C031952195310927
:1011B00094E0220F331F9A95E1F72E173F070CF4A6
:1011C000F901EE0DFF1DE11591E0F90710F0EFEFC9
:1011D000F0E02E2F2095382F320F08F43FEF832FA9
:1011E0000F91FF90EF900895EF92FF920F93970168
:1011F00095E0099F200D311D1124211591E039073B
:1012000010F02FEF30E02095382F320F08F43FEF29
:10121000832F0F91FF90EF9008950F931F93A42FAA
:1012200010E0F801EE0FFF1FEA57FB4F9081905737
:1012300097FD9195000F111FF801EA5AFB4F01A984
:101240000052110B2003A001219F500D112428E30F
:1012500030E0291B310997FD33951A2F1203F00155
:10126000139FF00D11244E0F5F1F9A01220F331FA1
:10127000240F351F37FF02C021583F4F220F232F65
:10128000221F330B620F1F910F9108950F931F932D
:10129000522F10E0F801EE0FFF1FEA5AFB4FA1A9F1
:1012A000A052BB0B9D015203F001539FF00D11247E
:1012B000000F111FD801AA57BB4F2C912057330B99
:1012C0004203D001439FB00D11249F012A0F3B1F01
:1012D00037FF02C0215C3F4F96E0359527959A95E0
:1012E000E1F7620F1F910F9108950F931F93522FF3
:1012F00010E0F801EE0FFF1FEA5AFB4FA1A9A05220
:10130000BB0B9D015203F001539FF00D1124000F00
:10131000111FD801AA57BB4F2C912057330B420302
:10132000D001439FB00D11249F012A0F3B1F37FFAF
:1013300002C021583F4F220F232F221F330B620F71
:101340001F910F910895EF920F931F9310E0980152
:10135000220F331F200F311F359527956E2D620FF9
:101360001F910F91EF900895322F50E0FA01EE0F88
:10137000FF1FEA5AFB4F91A9905297FD9195440F98
:10138000551FFA01EA57FB4F2081231B330B290F0E
:10139000311D97FD3A95620F0895E42FF0E0EE0FAE
:1013A000FF1FEA5AFB4F61A9621B0895E42FF0E08A
:1013B000EE0FFF1FEA57FB4F6081621B0895622FFB
:1013C000089508950F931F93CF93DF938B01D82F28
:1013D000C92F20E030E0A9010E94A65E81110AC059
:1013E000809190008F7380939000DF91CF911F9137
:1013F0000F91089580919000806880939000C801BB
:10140000AD2FBC2F8093980890939908A0939A08C9
:10141000B0939B0820E030E040E051E4B8018D2F0C
:101420009C2F0E94285D9B01AC0160E074E284E780
:101430009BE40E94F05D8B01D82FC92F0E94AF5E04
:10144000462F572F509397004093960060910602C5
:1014500070E080E090E00E945A5E98014D2F5C2F72
:101460000E94285D20E030E048EC52E40E94F05DEC
:101470000E94AF5E462F572F5093990040939800DB
:10148000B4CFE1E7F0E080818D7F8083E0E9F0E098
:1014900080818F7380830895EFE6F0E080818D7FF7
:1014A0008083E0E8F0E080818F7380830895982F37
:1014B000282F207F203D41F180F4203B31F038F48B
:1014C000907E903811F0203AD1F483E0089581E0C5
:1014D000203C09F080E0880F0895203EB1F3203FC2
:1014E00071F4833F89F020F4813F71F0823FECCFAB
:1014F00081E09D3F30F4983F30F4963F21F080E04A
:1015000008959E3FE0F3089582E00895FC019B0159
:10151000009719F4832F80780895AC0197FF04C0D9
:1015200044275527481B590BB901640F751F37FD18
:101530000FC0C901841B950BA5E0880F991FAA95C0
:10154000E1F70E944A5F80E2861BF7FD81950895CE
:10155000CB0165E0880F991F6A95E1F7BA01621B1C
:10156000730B0E944A5F80E6EFCFEF920F93CF9309
:10157000DF93D72FC82FBA01C9010E19C7DF602F1B
:10158000681B7D2F8C2FDF91CF910F91EF900895E5
:101590000F93CF93DF93D72FC82FBA01C901B6DFBE
:1015A000682F600F7D2F8C2FDF91CF910F910895C1
:1015B0009091450A982B9093450A0895A3C40895E5
:1015C000EFECFBE0808191E0892780831092690233
:1015D00081E0EECF8091CF0B8370811102C0109219
:1015E00069028091CF0B8C7F81608093CF0B08952F
:1015F0008091CF0B83708111109269028091CF0B83
:101600008C7F8093CF0B0895982F862F2091CF0B3E
:101610002370211581F0911579F09E3278F49F7333
:10162000990F990F2091CF0B2370922B9093CF0B92
:1016300010926902BDCF089591E0F2CF9DE2F0CF04
:101640008091CF0B869586958F5F8E3208F081E072
:1016500061E0DACF8091CF0B869586958A9509F463
:101660008DE261E0D1CF982F822F2091CF0B237094
:10167000211539F09093D00B6093D10B4093D20B8E
:1016800097CF0895EFECFBE0818190E021E043816A
:1016900062810896E8CFEFECFBE0818121E0438195
:1016A00062818850990BDFCFEFECFBE0628120E193
:1016B000620F08F46FEF818121E0438190E0D3CF86
:1016C000EFECFBE0628120E1621B08F460E08181C5
:1016D00021E0438190E0C7CFEFECFBE0438120E1C4
:1016E000420F08F44FEF818121E0628190E0BBCF8F
:1016F000EFECFBE0438120E1421B08F440E08181F4
:1017000021E0628190E0AFCFEFECFBE0248130E19B
:10171000230F08F42FEF248381E04ACFEFECFBE0A6
:10172000248130E1231B08F420E0248381E040CFB2
:1017300081152CE7920741F42091DF0B3091E00BEB
:10174000232B11F480E090E00895E2ECFFE080E0CC
:1017500090E061E77BE447E95BE42BE03CE47783DE
:1017600066835187408733872287978786870196CC
:1017700070968032910599F70895FB01811520E25A
:10178000920728F4811541E0940738F408959C01EC
:1017900030522115304348F00895392F94FF02C08C
:1017A0003295307F2081232B208399270895462B63
:1017B00022FF0FC0982F92959F708F70892B962FC4
:1017C00092959F706F70692B942F92959F704F70B8
:1017D000492B982F9623961309C050E040955095B9
:1017E00090E04823592381E0452B09F080E00895DB
:1017F00080913A1390913B1390935D0280935C0229
:101800000895EF92FF920F931F93CF93DF93FB0105
:101810008FEF9FEF4430510508F45FC04091621391
:1018200041FB882780F990E0880F991F42FB002731
:1018300000F910E0000F111F000F111F802B912BDA
:1018400040FBEE24E0F8F12C8E299F2943FB222750
:1018500020F9C22F50E0D52F53E0CC0FDD1F5A9551
:10186000E1F78C2B9D2B44FB222720F950E1259F8B
:1018700090011124822B932B45FB222720F950E263
:10188000259F90011124822B932B46FB222720F9C0
:1018900050E4259F90011124822B932B47FB222794
:1018A00020F940E8249F90011124822B932B209152
:1018B0006313322F3170932B26952170B22FBB0FFB
:1018C000A0E08A2B9B2B092E000CAA0BBB0B80835C
:1018D0009183A283B38380E090E0CDB7DEB7E6E0EA
:1018E0000C943B5F1092CA121092C912E1EEF1E122
:1018F0008581811102C014821682379682E1E13C13
:10190000F807B1F70895AC013091CC126091CB1279
:10191000232F621301C00895822F90E0FC01EE0F87
:10192000FF1FEF53FD4E0190F081E02DE417F50706
:1019300091F467E0649FF001659FF00D1124EF5171
:10194000FE4E41E044832313E6CF0196837099272E
:101950008093CC1208950196282F2370DACFFC01D2
:101960008481862381110AC082818115B9F06823A0
:10197000908593FF05C081E061110FC080E008955C
:10198000282F22952F708F70282B962F92959F705D
:101990006F70962B81E02913F1CF089581E00895AF
:1019A0000F931F93CF9301E010E0082E01C0000FAA
:1019B0000A94EAF7C091D5119C2F9023911115C07C
:1019C0009091DE11969596959695891306C0109282
:1019D000DE111092E0111092DF1197D8C027C0934A
:1019E000D511CF911F910F91089599D8F7CF90916C
:1019F000A10D89029001112437FF03C08093A10D2E
:101A000008952F3731051CF4980F9093A10D089578
:101A10009C0180E090E0F901E80FF91FE491E413E4
:101A200007C091E08927F901E80FF11D849108951D
:101A30000196861780F380E00895FA01309709F047
:101A400009950895A3E0B0E0E8E2FDE00C94235F7F
:101A50009C018091C0059091C10582179307B1F058
:101A60003093C1052093C005E091080CF091090C5A
:101A7000309761F00084F185E02D309739F083E0F4
:101A800089833B832A83CE01019609952396E2E060
:101A90000C943F5FA3E0B0E0E0E5FDE00C94235F31
:101AA0009C018091BE059091BF0582179307B1F00C
:101AB0003093BF052093BE05E091080CF091090C0E
:101AC000309761F00084F185E02D309739F084E0A3
:101AD00089833B832A83CE01019609952396E2E010
:101AE0000C943F5F90917802913091F0A8E9B5E0B5
:101AF000EFEF90E02D91821751F0EF3F19F4211193
:101B000001C0E92F9F5F9630A9F7EF3FC9F4089510
:101B10009091621397FFEACFE82FE695E695E69558
:101B2000803FA8F7F0E0E256FA4F877021E030E0FE
:101B300001C0220F8A95EAF78281822B8283089561
:101B40000E2E000CFF0BEA56FA4FF8CF0E941A5ADD
:101B500088E19CE00FB6F894A895809360000FBED2
:101B600090936000FFCFFC01462F878190850097FE
:101B700029F46581808191810C943D5A0895FC017E
:101B80006081718184E090E00C944F6090916313C8
:101B900092FB222720F9281749F080FB92F99093B5
:101BA000631382E693E1EBDF82E061C808951F933F
:101BB000CF93DF93962F122F632F8830D8F4943071
:101BC000C8F44C30B8F4C42FD0E0CC0FDD1F28E1AE
:101BD000929FC00DD11D112490E6899FC00DD11D8B
:101BE0001124CE0189960E943560612FCE018A961C
:101BF0000E943560DF91CF911F9108956091B60DDD
:101C000061606093B60D87E090E00E94356062E00D
:101C100070E088E192E00C94605781E08093D00DF1
:101C200068E070E084EC91E00C94605781E0809370
:101C3000CF0D68E070E084E491E00C946057A7E079
:101C4000B0E0E5E2FEE00C94205F8C0108511F4FEC
:101C50008091E10B843009F063C0809170028F7035
:101C60008093E9008091E80082FF5AC08091E800EB
:101C700085FF56C040E050E064E070E0CE01019680
:101C80000E94E9528091E80085FD05C08091E8003E
:101C90008B778093E800FA808F2D09DC282FFD8256
:101CA0008B818E838C818F83211108C0E981E45060
:101CB000E43070F6F0E0EE50FC4F208130E0321757
:101CC00038F6FE013596E30FF11DF0804FB7F8941A
:101CD000D8011196EC911197F0E0CF010196129680
:101CE0006C9170E00E944A5FD8015C915817190608
:101CF00019F44FBF3F5FE3CF13968D919C911497DA
:101D0000E80FF91FF08211968C91119790E00196DF
:101D100012966C9170E00E944A5FF8018183E9CFCE
:101D20002796E5E00C943C5F0F931F93CF93DF93CE
:101D30000AE313E1C9E2D3E0CE010E941960F80181
:101D400061918F01681719F0CE010E9435602196CC
:101D5000C135F3E0DF0781F7DF91CF911F910F913C
:101D600008950F931F93CF93DF930AE313E1C9E222
:101D7000D3E0CE010E941960F80181938F01219672
:101D8000C135F3E0DF07A9F7C6EED3E0FE01859188
:101D90009591009711F0FC0109952C96F4E0C23B57
:101DA000DF07A1F7DF91CF911F910F9108950F9356
:101DB0001F93CF93DF93883030F5643020F54C309B
:101DC00010F5C42FD0E0CC0FDD1F28E1629FC00DBD
:101DD000D11D112430E6839FC00DD11D1124CE01E9
:101DE00089960E941960082F10E0102F0027CE015D
:101DF0008A960E9419609801282BC901DF91CF9122
:101E00001F910F91089580E090E0F8CF382F292F8F
:101E1000CB01A32FB22F8F3228E09207A105B10585
:101E200020F48F52984F0C94196080E0089585E259
:101E300090E00E941960813789F486E290E00E9468
:101E400019608B3B59F487E290E00E94196091E0A1
:101E50008F3209F090E0892F8170089580E0FCCFE7
:101E6000A4E0B0E0E6E3FFE00C94205FFC01F62E76
:101E7000042F122FC19708F041C0EE0FFF1FEE0F85
:101E8000FF1FBF01685E7D4F44E050E0CE01019628
:101E90000E94D25F89818370AA814A2F50E02B81F2
:101EA00030E0EC81F0E064EA869FC0011124BC01BF
:101EB0006C5B784FA60FB72FB11DAC91AF110CC062
:101EC000DB01A20FB31FAC91A01306C0DB01AE0F64
:101ED000BF1F6C91611791F08C5B984FDC01A40FD0
:101EE000B51FFC92280F391FD9010C93E80FF91F79
:101EF000108380579F4F21E0FC0120832496E5E06A
:101F00000C943C5FFF920F931F93CF93DF93182F96
:101F1000062FF42EC0E0D0E02F2D402F612FCE01F0
:101F20009FDF2196C133D105B9F7CDB7DEB7E5E024
:101F30000C943C5FAAE0B0E0E0EAFFE00C941D5F87
:101F4000E4EEF5E080E491E0DF019C011D92215078
:101F50003040E1F7E1EEF1E180EEDF011D928A957C
:101F6000E9F784EEC82E85E0D82E7F0101E914E060
:101F7000F701D182C0824AE050E0B801CE0101965B
:101F80000E94096088E0FE013196D60101900D9211
:101F90008A95E1F789859A85D70113969C938E934C
:101FA0001297BAE0CB0ED11CE7E0EE0EF11C065FF3
:101FB0001F4F013DF5E01F07D9F62A96E8E00C9483
:101FC000395FAAE0B0E0E7EEFFE00C941B5F07ED9D
:101FD0001DE081EDE82E85E0F82E97E0B92E23EE86
:101FE000C22E25E0D22EAA24A3944AE050E0B701E5
:101FF000CE0101960E940960F8013896DF018B2D11
:102000001D928A95E9F789819A81D80111969C934E
:102010008E938F8112968C9312978D8113968C9349
:102020001397888514968C931497898515968C93AD
:1020300015978B819C8117969C938E9316978A8512
:1020400087FD04C01E96DC92CE921D9780FF02C0D1
:10205000F801A08681FF07C0D80118969C911897B7
:10206000926018969C9382FF04C0F801908594605A
:10207000908783FF07C0D80118969C9118979860A5
:1020800018969C9384FF04C0F80190859061908716
:1020900085FF07C0D80118968C9118978062189612
:1020A0008C93BAE0EB0EF11C015F1F4FE1E1EE16DD
:1020B000E7E0FE0609F099CF2A96EAE00C94375F34
:1020C000A6E0B0E0E6E6F0E10C941E5F06E91CE055
:1020D00081E1E82E87E0F82E98E0D92E46E050E026
:1020E000B701CE0101960E940960F8018D2D119271
:1020F0008A95E9F7B8016C5F7F4F89819A813DDB52
:10210000F80191838083B8016B5F7F4F8B819C8145
:1021100034DBF801938382838D8186838E8187836C
:10212000F6E0EF0EF11C085F1F4F81EDE81687E027
:10213000F806A1F62696E7E00C943A5F9C01CB01E5
:10214000BA01F9013296E4914E2F50E06E177105F5
:1021500048F0F9013496659175910E94E85F80E03E
:1021600090E008958FEF9FEF0895A4E0B0E0EBEBCF
:10217000F0E10C94205F8B01FC013396F4901982FE
:102180001A821B821C82452B31F48FEF9FEF24961D
:10219000E5E00C943C5F44E050E0BE016F5F7F4F90
:1021A000CDDF019691F381E090E00F2C02C0880F03
:1021B000991F0A94E2F7092E000CAA0BBB0B498168
:1021C0005A816B817C8184239523A623B72321E048
:1021D000892B8A2B8B2B09F420E0F801208380E0E7
:1021E00090E0D5CF9C01CA01F9013296E4914E2FBF
:1021F00050E08E17910550F0F90134968591959134
:102200000E94E85F91DD80E090E008958FEF9FEFFE
:102210000895A4E0B0E0EFE0F1E10C941C5F7C01D4
:102220006B01CA01F7013396B49019821A821B829E
:102230001C82892B31F48FEF9FEF2496E9E00C94F8
:10224000385F44E050E0BE016F5F7F4FC70176DF2B
:10225000019689F381E090E00B2C02C0880F991F52
:102260000A94E2F780959095092E000CAA0BBB0BFF
:1022700049815A816B817C8184239523A623B723CE
:10228000F6012081022F017010E00B2C02C0000F1C
:10229000111F0A94E2F7012E000C220B330B802B46
:1022A000912BA22BB32B89839A83AB83BC8344E00D
:1022B00050E0BE016F5F7F4FC70194DFBECFA4E047
:1022C000B0E0E5E6F1E10C941E5F7B01142FD22E05
:1022D0004A832B830C83842FEAD881113BC082E090
:1022E000E816F10489F083E0E816F10441F081E09A
:1022F000E816F10459F12496E7E00C943A5F17E0F0
:10230000073F31F014E004C087EF16E0D812FACF8F
:1023100019838091E10B843071F780916B028F708B
:102320008093E90040E050E064E070E0CE01019667
:102330000E9477528111DFCF8091E80085FDDBCFCD
:102340008091E8008E778093E800D5CF173FD1F6D3
:1023500015E0DECF12951F70DBCF48E050E067E15B
:1023600070E08FEC9BE00E9426601092450A089571
:10237000EFECFBE085E380838091B9039091BA0391
:10238000A091BB0381839283A3838FE784838FEF24
:102390008583E3CFA0E1B0E0E0EDF1E10C94155FBF
:1023A000FE01319680E1DF011D928A95E9F703E88D
:1023B00010E091EDA92E97E0B92E2FE2422E28E0F1
:1023C000522E612C712C4F0173016201B1E14B1649
:1023D0005104610471041CF080E1C82ED12CA601C7
:1023E000B501C4010E942660AC0CBD1C0D2C000C74
:1023F000EE08FF084C185D086E087F080150104079
:1024000019F76096E0E10C94315FA1E0B0E0EBE0F9
:10241000F2E10C94215F4983E82FF0E0E851FC4F92
:10242000808104E610E021E030E0AE014F5F5F4FB5
:10243000880F0E94E55A2196E4E00C943D5FA3E0EA
:10244000B0E0E5E2F2E10C941D5F84ED97E09B8340
:102450008A8388EEE82E83E0F82EEA81FB81808172
:102460008115D9F0E059F1096F0124E22983F701C0
:10247000808104E610E020E130E0A6016981880F48
:102480000E94E55AF981F05FF98320E1C20ED11C68
:10249000F43B69F7EA81FB8110828A819B818C552C
:1024A0009F4F9B838A839FEFE91AF90AEA81FB8198
:1024B000EC51F94091F62396E8E00C94395FA4E0E2
:1024C000B0E0E5E6F2E10C941D5F0E94AF5A10E027
:1024D0004BE06DEF812F99DF40E06AE0812F95DFBF
:1024E0008FE39CE90197F1F700C0000040E060E055
:1024F000812F8BDF40E061E0812F87DF40E066E0E5
:10250000812F83DF40E06DEF812F7FDF00E040E02F
:10251000602F812F7ADF0F5F0231C9F740E0602F13
:10252000812F73DF0F5F0432C9F740E0602F812FE6
:102530006CDF0F5F043BC9F74BE06DEF812F65DF68
:1025400041E06AE0812F61DF40E06DEF812F5DDFC8
:1025500081E0810F11E0823009F0BACF08E112E08A
:1025600024EAC22EEE24E394F12CDD24D39444E03B
:1025700050E0B801CE0101960E94D25F6A814B8182
:102580002C8189818370E62FE695E695E695C89EB5
:10259000C00111248C5B984FE80FF92FF11DEF5605
:1025A000FF4F6770D70102C0AA0FBB1F6A95E2F701
:1025B00030813A2B3083E42FE695E695E695E80FD7
:1025C000F92FF11DEF56FF4F4770B70102C0660F9C
:1025D000771F4A95E2F73081362B3083E22FE6955C
:1025E000E695E695E80FF92FF11DEF56FF4F27709E
:1025F000D70102C0AA0FBB1F2A95E2F79D013081C7
:10260000232B20838D559F4FFC01D0820C5F1F4FE1
:10261000F2E00C3D1F0709F0AACF8091E707811572
:1026200081F095EDE92E97E0F92E10E0D7014D915C
:102630007D01612F80E0E9DE1F5F1231B9F7109252
:10264000E70780918B08811581F089E7E82E88E003
:10265000F82E10E0F70141917F01612F81E0D5DE76
:102660001F5F1231B9F710928B082496E8E00C94A2
:10267000395F9C012115310509F408958FE99FE028
:102680000197F1F700C0000021503109F3CF292F45
:10269000943090F58C3080F590E03CE0239F800DE5
:1026A000911D1124282F277041E001C0440F2A9565
:1026B000EAF723E0969587952A95E1F7FC01EE0F5E
:1026C000FF1FE80FF91FE559F34F20E030E070E0FD
:1026D0005191DF01CB01022E02C0969587950A9495
:1026E000E2F7817081958527842385278E932F5F5C
:1026F0003F4F2330310561F70895292F943078F545
:102700008C3068F590E03CE0239F800D911D1124F2
:10271000682F677023E0969587952A95E1F7FC016D
:10272000EE0FFF1FE80FF91FE559F34F40E050E0AF
:1027300080E0219130E0062E02C0369527950A945C
:10274000E2F721703327042E01C0220F0A94EAF722
:10275000822B4F5F5F4F4330510559F7089580E05A
:102760000895982F90958091DA1189238093DA113A
:102770000895462F672F2091E40B3091E50B232B12
:1027800081F4703F39F4403F61F48091E20B909105
:10279000E30B0895743028F44C3018F4883008F4B2
:1027A00006CB80E090E00895A0E0B0E0EAEDF3E130
:1027B0000C941E5F7C010091391380913813082B13
:1027C000C7E0D0E010E0C8010C2E02C095958795B7
:1027D0000A94E2F780FD09C02197A8F7D12C8D2D2E
:1027E000CDB7DEB7E7E00C943A5FDC2EB7018C2F53
:1027F000C0DF0E945E07019779F3F1CFCF93DF939B
:10280000D82FC92FD1DF6D2F7C2FB3DF0E945E0739
:10281000DF91CF910895FC018481811561F087815A
:102820009085009721F00E945E070C945B058081E3
:102830009181E4DFFACF80E00895F894E82FE295E3
:10284000EF70F0E041A18F7021E030E0B90102C0EB
:10285000660F771F8A95E2F7CB01962F9095942308
:1028600091A392A1892B82A3789408958091070265
:10287000811124C01092A5080E94410A0E944C0AAE
:102880001092A4081092A3081092A2081092A10816
:10289000E6EAF8E080E090E0A0E8BFEB1182108269
:1028A00082839383A483B58317821682389628E0A7
:1028B000E63EF20799F781E0809307020895809140
:1028C000E608811137C087E090E00E94196080938C
:1028D000B60D82FD08C0682F67606093B60D87E073
:1028E00090E00E943560E6EAF8E080E090E0A0E841
:1028F000BFEB1182108282839383A483B5831782F6
:102900001682389628E0E63EF20799F70E94410ABF
:102910003E9A0E944C0A259A92E0909390008AE198
:1029200080939100909380008093810081E0809358
:10293000E6089CCF0895A0E0B0E0E1EAF4E10C9451
:102940001D5F6B017C0120E030E0A901C701B601E9
:102950000E94A65E87FF04C0F7FAF094F7F8F0949F
:102960008091A308811509F458C08091E60881116F
:1029700001C0A5DF06EA18E0C7E0D0E0A701960194
:10298000F80162AD73AD84AD95AD0E94A65E811174
:102990003DC0CE0123E0880F991F2A95E1F78A55A3
:1029A000974FF8E08E3D9F0739F51092DF0810929F
:1029B000DE0880E090E0A0E8BFEB8093E008909311
:1029C000E108A093E208B093E3081092E5081092A2
:1029D000E408C1E0C093A0088091A50881508093CD
:1029E000A50881111AC00E94410A0E944C0AC09396
:1029F00007021092A30811C028E0FC013896DC0100
:102A000001900D922A95E1F70896CBCF21970850B7
:102A10001109CF3FDC0709F0B1CFCDB7DEB7E8E051
:102A20000C94395F0F93CF93C82F8091D00D8115EF
:102A3000F9F08C2F8554990BBC01072E000C880BE4
:102A4000990B0E945A5E20E030E040E451E40E947D
:102A5000F05D9B01AC0160E070E080E090E40E94DA
:102A6000C75B20E030E04CED53E40E94285D63DF5B
:102A70008091CF0D811569F02C2F2F77E0914B0AB3
:102A8000F0914C0A00E040E863E070E08BE49AE0EB
:102A90000995CF910F91089562E070E088E092E08F
:102AA0000E9460572FEF81EE94E0215080409040CB
:102AB000E1F700C00000DADE6091B60D6E7F609332
:102AC000B60D87E090E00C9435600F93E0914B0ACF
:102AD000F0914C0A00E02BE740EB63E070E08BE400
:102AE0009AE009950F910895F0DF1092CF0D68E0FC
:102AF00070E084E091E00C946057CF92DF92EF9207
:102B0000FF921F93CF93DF93172FE82FF0E0E4524B
:102B1000FD4F71110CC0E4918E2F7E2F6E2FDF912F
:102B2000CF911F91FF90EF90DF90CF900895E62E08
:102B3000F12CC72ED12CF491EF2F86E0689F9001E5
:102B40001124CFEFD0E0C901BE010E94FF5EAB01AE
:102B5000EE0CFF1C65E5649FC001659F900D11247C
:102B6000E81AF90A6E2D660F6E0D7E01EC18FD084D
:102B7000FE9DD001FF9DB00D11248B2F169F70017B
:102B80001124EF2CFF246E01CE18DF087601FE9D84
:102B90006001FF9DD00C11247E01E61AF108B701F7
:102BA000169F7001179FF00C1124EF2CFF24CE19F3
:102BB000DF09FC9F7001FD9FF00C11247F2D433035
:102BC0005105C1F02C3F334058F441305105B1F06C
:102BD0004230510509F0A2CFEB2F8F2D7F2F9ECFD2
:102BE0004430510571F04630510509F497CF7B2FE1
:102BF0008D2D94CF7D2DEB2F8F2F90CF7F2FED2D0F
:102C00008DCFEF2D7B2FF8CF282F269F020E20E0AF
:102C1000211D1124822F08951F93CF93DF93162F28
:102C2000D72FC82F60E4842F8095EEDF682F610FC7
:102C30007D2F8C2FDF91CF911F910895CF93DF933C
:102C4000D62FC72F682F842F8095DEDF6D2F7C2F26
:102C5000DF91CF9108951F93CF93DF93162FD72F36
:102C6000C82FE42FF0E0EE0FFF1FEA57FB4F8081E3
:102C7000821B87FD819568E1C7DF682F610F7D2F7B
:102C80008C2FDF91CF911F910895EF920F931F9397
:102C9000CF93DF93162FD72FC82FBA01C9010E1972
:102CA0000C0F0E94860A6C2F081B802FADDF612F4E
:102CB0007D2FDF91CF911F910F91EF900895EF92AB
:102CC0000F931F93CF93DF93162FC72FD82FBA01DF
:102CD000C9010E190C0F0E94860A6C2F081B802F49
:102CE00093DF782F612F8D2FDF91CF911F910F915F
:102CF000EF9008950F931F93CF93DF93162FD72F45
:102D0000C82FBA01C9012C2F201B022F0E94860A4E
:102D1000982F990F990F891B6C2F800F75DF612FEA
:102D20007D2FDF91CF911F910F9108950F931F93E6
:102D3000CF93DF93162FC72FD82FBA01C9012C2F9D
:102D4000201B022F0E94860A982F990F990F891B2A
:102D50006C2F800F59DF782F612F8D2FDF91CF914E
:102D60001F910F9108950F931F93CF93DF93162F09
:102D7000D72FC82F022FE42FF0E0EE0FFF1FEA57E6
:102D8000FB4F64EE808140DF6C2F70E0482F50E0F5
:102D9000445E5F4F202F30E0CA01801B910997FFEE
:102DA00003C0C901841B950B23E0880F991F2A9546
:102DB000E1F79B01281B390BC90137FF02C080E0F6
:102DC00090E06C2F21DF612F7D2FDF91CF911F913C
:102DD0000F9108950F931F93CF93DF93162FC72F53
:102DE000D82F022FE42FF0E0EE0FFF1FEA57FB4F22
:102DF00064EE808109DF6C2F70E0482F50E0445E64
:102E00005F4F202F30E0CA01801B910997FF03C05C
:102E1000C901841B950B23E0880F991F2A95E1F7C0
:102E20009B01281B390BC90137FF02C080E090E0ED
:102E30006C2FEADE782F612F8D2FDF91CF911F91BC
:102E40000F9108959C0180E090E0269F020E811D65
:102E5000369F800D911D1124830F911D089520919F
:102E6000D30B30E1230F08F42FEF60E1822F90E0C5
:102E7000E9DFBC0188EB9BE00E94FF5E80E090E010
:102E800008959C018230910508F408959FEF213E3A
:102E90008EE1380740F4C90145E0969587954A953B
:102EA000E1F798E0980F61E0E62FE90FFF27FF1F99
:102EB000AF0155954795842F449FF001459FF00D34
:102EC000F00D11242E173F0738F49FEF940F96173B
:102ED00058F78FEF860F08954F3FE9F361E0640FD5
:102EE000F6CF0F93CF93DF93D72FC82FB90147FDAC
:102EF000419528E330E0241B310947FD3395229F9B
:102F0000A001239F500D500D1124669FC001679FA3
:102F1000900D900D1124840F951FB3DF982F990FFA
:102F2000692F680F600F7D2F8C2FDF91CF910F914C
:102F30000895409104025091050225E038E0429F37
:102F4000C001439F900D529F900D1124875E994CB4
:102F50009093050280930402890F0895CF93C82FA0
:102F6000E8DF8C9FC0011124892FCF910895982FFD
:102F7000E82F96FDE0958E2F8F7096FD8F5FE6957A
:102F8000E695E695E670F0E0E651FC4F2181289F3A
:102F9000202D812D112422952F708295807F282B42
:102FA0008081820F97FD8195805808950F931F931C
:102FB000CF93DF938B01D82FC42F822FD8DFEC2F34
:102FC000F0E0EE0FFF1FEA57FB4F90819058890FFA
:102FD00087FD81956CE0880F17DE682F600F712FD9
:102FE0008D2FDF91CF911F910F9108951F93CF9354
:102FF000DF93162FD72FC82F822F8695B8DF8058E2
:1030000087FD81956CE0880FFFDD682F610F7D2FB4
:103010008C2FDF91CF911F9108951F93CF93DF9352
:10302000D62FC72F182F822F8695A1DF805887FDB6
:103030008195612F880FE8DD6D2F7C2FDF91CF9177
:103040001F9108950C94300F08959AE0899F802D68
:103050001124980F923308F091E30895AC0123E016
:10306000969587952A95E1F78E719927FC01ED5386
:10307000FA4F0190F081E02D4F70552721E030E0AC
:1030800002C0220F331F4A95E2F7611541F0E22B8F
:10309000F32B8D539A4FDC01ED93FC93089520950B
:1030A0003095E223F323F5CF282FCB01203270F4A3
:1030B0004AE0249F90011124B9016F5A7C4F4AE0E5
:1030C00050E00E94096080E090E008958FEF9FEF4C
:1030D0000895CF92DF92EF92FF92CF93DF93D82F94
:1030E000C92FC090BC0FD090BD0FE090BE0FF090E4
:1030F000BF0F0E946F4D6C197D098E099F09643FB7
:1031000071408105910518F10E946F4D6B017C01A2
:1031100082E390E0A0E0B0E0C092FE08D092FF0809
:10312000E0920009F09201098093FA089093FB085D
:10313000A093FC08B093FD08D093BA0FC093BB0FC7
:10314000DF91CF91FF90EF90DF90CF90089584EFC3
:1031500091E0A0E0B0E0E0CF8091D00D811186DB5E
:103160008091CF0D8111B1CC0895F6DF1092D00D72
:1031700068E070E084E891E00C946057E091080CFE
:10318000F091090C309739F00190F081E02D3097E3
:1031900011F00995089580E00895F0DF909167138C
:1031A000981721F0809367130C946F4D08958091C8
:1031B0003C1390913D13892B91F00E945A4D209120
:1031C000D6113091D711AC01421B530B9A0181E00B
:1031D00040913C1350913D132417350708F480E0CB
:1031E0000895CF93DF93C091DA118091DD11C82B40
:1031F0008091D8118115F1F080913C1390913D138D
:10320000892B21F0D4DF81110E946006D091D81162
:1032100080917802813021F48091621387FD14C07F
:1032200086E028E935E090E0815090F491110E9409
:103230006006CD2B8091D60D80958C239091D50D75
:10324000892BDF91CF9108958EE120EA35E0EBCF15
:10325000F90141919F01411539F39F5FE5CF8091BD
:103260007802813061F58091621387FF28C0B9DF51
:1032700080939F0540E250E068EE7BE08EE995E0A8
:103280000E94DB5F892BD1F080E2EEE9F5E0A8EE49
:10329000BBE001900D928A95E1F7E091080CF09166
:1032A000090C309759F00480F581E02D309731F00A
:1032B00086E080939E058EE995E00995089591DF5B
:1032C0008093960548E050E06AE07CE086E995E06E
:1032D0000E94DB5F892B91F388E0E6E9F5E0AAE044
:1032E000BCE001900D928A95E1F7E091080CF09115
:1032F000090C309719F30280F381E02D3097F1F239
:1033000086E995E0DACF811519F00E945206A7CF21
:103310000895811531F09091DD11892B8093DD1195
:103320009ECF0895811511F01CDA99CF089581156B
:1033300019F00E94580693CF08958091D10D811500
:1033400021F082E2F4DF1092D10D0895CF93C82FBF
:103350008115B1F08238B1F411DF81FD11C089E32C
:103360000E94720D7CDF2FEF37EE83E0215030405A
:103370008040E1F700C0000089E30E940B4D6FDF41
:10338000CF910895833891F4F9DE80FDF9CF83E57C
:103390000E94720D64DF9FEF21EE34E091502040D7
:1033A0003040E1F700C0000083E5E7CF843891F4B6
:1033B000E5DE82FDE5CF87E40E94720D50DF8FEFDE
:1033C00091EE24E0815090402040E1F700C00000E1
:1033D00087E4D3CF8CEF8C0F813A88F58091780207
:1033E000813071F0E8E9F5E08EE995E02191C217AE
:1033F00009F18E179F07D1F78C2F0E94720DBFCF56
:103400008091621387FFEECFEC2FE695E695E69567
:10341000F0E0E256FA4F828190E04C2F477021E0B5
:1034200030E002C0220F331F4A95E2F78223932334
:10343000892B11F38C2F0E940B4D11DFDDCF80E221
:103440008C0F883048F4C77081E001C0880FCA959E
:10345000EAF70E94520693CF8BE58C0F833038F445
:103460002C2F2452330BC9010E94220D89CFC85A38
:10347000CB3108F085CFEC2FF0E0EE0FFF1FE15BC2
:10348000FA4F808191810E944A0D7ACFCF93DF93CA
:10349000EC01805E9109089720F069E879E12097B6
:1034A00011F463E879E1CE010E943C058C2F4EDFD8
:1034B000DF91CF910895811509F443C0823859F402
:1034C0005DDE81FF3EC089E30E94720DC8DE89E3A4
:1034D0000E940B4DC4CE833849F450DE80FF31C0CA
:1034E00083E50E94720DBBDE83E5F2CF843849F498
:1034F00045DE82FF26C087E40E94720DB0DE87E4BD
:10350000E7CF9CEF980F913A18F390E2980F98301C
:1035100048F4877091E001C0990F8A95EAF7892FE6
:1035200020D9D8CF9BE5980F933020F480E090E02D
:103530000C94220D885A8B3120F480E090E00C949A
:103540004A0D0895CF93DF93EC01B5DFCE01805E85
:103550009109089720F067E979E1209711F462E971
:1035600079E1CE010E943C05DF91CF9108951F9330
:10357000CF93DF93182FEB01E9DE209731F4812FF1
:103580009ADFDF91CF911F9108958FE99FE0019716
:10359000F1F700C000002197F0CF60915A137091AD
:1035A0005B13893321F06091581370915913DFCF69
:1035B0001092DA11809178028130B1F48091621317
:1035C00087FF12C0E0EAF5E08EE1DF011D928A95E7
:1035D000E9F780E090E00E94220D80E090E00E94F8
:1035E0004A0D1092DD113BCEE8E9F5E086E0EDCF23
:1035F000CF93DF93D82FC92F2091220C283010F0C1
:10360000D7DF20E0E22FF0E0EE0FFF1FEE5EF34F7A
:10361000D083C1832F5F2093220CDF91CF91089537
:10362000CF93DF93FB018FEF9FEF4430510590F074
:10363000D081C181BDDFD0936213C37080916313C9
:103640008C7FC82BC093631382E693E10E94BF0D69
:1036500080E090E0DF91CF910895EAE3F3E1128EEC
:10366000138E8FEA90E09183808385E0848F28E831
:1036700033E13383228322E330E0378B268B28EC3F
:1036800030E0318F208F158E35A324A3178E168E30
:1036900020E530E031A320A382A317A216A20E9446
:1036A000940E86DF109263131092621380E08460A0
:1036B0008093631382E693E10E94BF0D0C94B10ED8
:1036C000AAE0B0E0E6E6FBE10C94185FC090DF0BE7
:1036D000D090E00B81E090E09093E00B8093DF0BC3
:1036E000812C912C10E0540100E01AC021E030E060
:1036F000143020F4F701859195919C01472D602F9E
:10370000812F0E94D70D739422E0E20EF11C3CE061
:103710007312ECCF0F5F8CE0A80EB11C043049F09F
:10372000C501880F991FFC01E856FF4F7F01712CDE
:10373000DDCF1F5FF0E38F0E911C1830A1F68DDFF7
:103740001A8219821C821B821E821D8218861F8289
:1037500088EC90E09A87898701E513E09E012F5F4E
:103760003F4F79014AE050E0B801C7010E94536021
:10377000065F1F4F013934E01307A1F78AE0F70114
:1037800011928A95E9F74AE050E0B801C7010E941A
:103790005360065F1F4F013DF5E01F07A1F789E069
:1037A000F70111928A95E9F78FEF9FEF9E838D8342
:1037B00087E08A874AE050E0B801C7010E94536061
:1037C000065F1F4F0131F7E01F07A1F786E0F70101
:1037D00011928A95E9F746E050E0B801C7010E94CE
:1037E00053600A5F1F4F013DF7E01F07A1F7D0921A
:1037F000E00BC092DF0B2A96EDE00C94345F6FEF84
:1038000085E290E00E9435606FEF86E290E00E94D2
:1038100035606FEF87E290E00E94356060E088E2FB
:1038200090E00E9435604CDF0E94CA1161E785E29A
:1038300090E00E9435606BEB86E290E00E9435607C
:103840006FE287E290E00C943560A2E0B0E0EBE23A
:10385000FCE10C94235F63EE7EEF80E090E00E9439
:103860004F6060E082E090E00E94356081E08093EC
:10387000381361E083E090E00E943560198284E1B2
:103880008A83CE0101960E94BF0D60E087E090E040
:103890000E9435600E94B811B2DF40E050E0BA01EA
:1038A0008FE090E00E94476040E050E0BA0183E181
:1038B00090E00E9447600E94AD112296E2E00C94D5
:1038C0003F5F80913F03877F80933F038091D10DBD
:1038D000811103C082E00E94580680913F0384FF5B
:1038E00006C08F7E80933F0382E00E945206809143
:1038F0003F0385FF06C08F7D80933F0380E20E94D7
:103900005206ADCCCF93DF93EC014A855B856E8583
:103910007F850E941D0D8B810E9458068C810E941C
:10392000B1139DDC86E0FE0111928A95E9F7DF91E3
:10393000CF910895CF93DF93EC018D8181FD13C06A
:1039400082608D838091DD119B81892B8093DD11B5
:103950008C810E94520683DC488559856E857F855F
:10396000CE010E941D0D1092C3111092C2118D81C3
:1039700080FD02C0CE01C6DFDF91CF910895962F62
:103980002091631322FF10C0682F660F660F660F29
:10399000692B6093DE110E9485050E945A4D909319
:1039A000E0118093DF1108950C9485059091D81152
:1039B000292F2823211561F0809589238093D81120
:1039C000811539F00E945A4D8093D6119093D711EA
:1039D000089580E090E0F8CFCF93C82F80916313D3
:1039E00082FF0CC08091D8118C1741F00E945A4D73
:1039F0009093D7118093D611C093D811CF91089589
:103A0000A0E0B0E0E6E0FDE10C941D5FE091A508C8
:103A10008E1708F042C2E150E81B48E0E402F001D2
:103A20001124EA55F74F02811381D481C58120E02A
:103A300030E0A901B8018D2F9C2F0E94A65E1816B8
:103A40000CF02BC2C0909E08D0909F080E945A4D47
:103A50007C01EC18FD08C70164E670E00E94FF5E7F
:103A6000E091B70DE93038F4F0E0E65FFE490C94E0
:103A70005D5F10929D0880919C08811591F10E94D4
:103A80005A4DBC0180E090E00E94585E20E030E09A
:103A900048E451E40E94F05D20E030E040EA51E467
:103AA0000E94385B0E94AA5E462F572F440F551F75
:103AB000440F551FFA01EA50FC4F608171818281E9
:103AC000938120E030E040E05FE30E94C75B9B0110
:103AD000AC01B8018D2F9C2F0E94285D8B01D82F3F
:103AE000C92FB8018D2F9C2FCDB7DEB7E8E00C941D
:103AF000395F10929D0881E080939C08BCCF1092A2
:103B00009D0850EDE51657E0F50648F488EEE816F6
:103B100083E0F80650F089E180930602ACCF64514F
:103B2000710988E1653B7105B8F38CE0F5CF10921F
:103B30009D0820E030E040EA52E4B8018D2F9C2F30
:103B40000E94A65E87FD97CF20E030E040E253E47C
:103B5000B8018D2F9C2F0E94A65E87FF2EC00E9469
:103B6000C45F68E270E00E944A5FBC01645C7F4F02
:103B7000072E000C880B990B0E945A5E8B01D82FE0
:103B8000C92F4BE0E416F10408F4ACC0C7010B9751
:103B90000A9718F0109206026ECF2EECA7012403AC
:103BA000C001259F900D1124865E9B4F6AE070E056
:103BB0000E94FF5E609306025ECF20E030E040EAA4
:103BC00053E4B8018D2F9C2F0E94A65E87FF27C06B
:103BD0000E94C45F68EE73E00E944A5FBC016851B6
:103BE0007C4F072E000C880B990B0E945A5E8B01AC
:103BF000D82FC92F56E0E516F10408F473C0C701A9
:103C000006970F9738F62EECA7012403C001259FD5
:103C1000900D1124865E9B4F6FE070E0C9CF20E0CD
:103C200030E040E254E4B8018D2F9C2F0E94A65E44
:103C300087FF28C00E94C45F60ED77E00E944A5F62
:103C4000BC016854744F072E000C880B990B0E941E
:103C50005A5E8B01D82FC92F50E1E516F10408F404
:103C600041C0C7014097059708F094CF2EECA701FB
:103C70002403C001259F900D1124865E9B4F65E0B3
:103C800070E096CF20E030E040EA54E4B8018D2F98
:103C90009C2F0E94A65E87FFEECE0E94C45F60ED5F
:103CA00077E00E944A5FBC016854744F072E000CF5
:103CB000880B990B0E945A5E8B01D82FC92F54E2B2
:103CC000E516F10478F0C70184970F9708F062CFEA
:103CD0002EECA7012403C001259F900D11248A50CA
:103CE000964F9ACF82E318CF81E080939D0850EDE4
:103CF000E51657E0F506B0F420E030E040E85EE37A
:103D000088EEE81683E0F80620F020E030E040E09E
:103D10005FE3B8018D2F9C2F0E94285D8B01D82F67
:103D2000C92F03CFCB014497853B910508F032CFD3
:103D300080E090E00E94585E20E030E040EA51E4EC
:103D40000E948B5D20E030E044E353E40E94F05D8C
:103D5000262F372F482F592F0E94285D20E030E072
:103D600048E451E40E94285D0E94AF5E8CE0861B0F
:103D7000D3CE81E080939D082AE0269FC001279F33
:103D8000900D112468EB7BE00E94FF5EBC016C5D2E
:103D9000754077FF03C071956195710970E080E00F
:103DA00090E00E945A5E2EE333EC4EE259E30E940B
:103DB000285D20E030E040EC5EE30E948C5D0E94D4
:103DC000AF5EF8CEC7018370992762E3892BD1F0EB
:103DD0006E2D6170772771956195710964767727EB
:103DE00080E090E00E94585E20E030E040E05EE33A
:103DF0000E94285D20E030E040E45FE30E948C5D9B
:103E00000E94AF5E81E080939D0847E0E422FF249A
:103E1000E114F10409F4BECECDCE81E080939D087B
:103E200082E3809306025CEFE5165AE3F50608F498
:103E300022CE80E090E00E94585E20E030E047E132
:103E400053E40E948B5D20E030E04AE754E40E9496
:103E5000F05D20E030E048E452E40E94285D20E07C
:103E600030E040EA51E40E94385B0E94AA5E462F8F
:103E7000572F440F551F440F551FFA01EA50FC4FAE
:103E80002081318142815381B8018D2F9C2F0E9466
:103E9000285D8B01D82FC92FEECD00E010E0D0E0D7
:103EA000C0E01FCEA0E0B0E0E8E5FFE10C94185FB1
:103EB0004B015C016A018091B60D80FF7CC080914E
:103EC000E608811102C00E945F1420E030E0A901E1
:103ED000C501B4010E94A65E87FF04C0B7FAB09482
:103EE000B7F8B0947090A508872D8150990B7C018C
:103EF0008C010F3F100709F049C0C1E0C70DC93060
:103F000008F477C088E08093A50848E350E06EEAA3
:103F100078E086EA98E00E94F15FC8E081E0809353
:103F2000A0088093A308C150DD0B0E945A4DFE01EA
:103F300023E0EE0FFF1F2A95E1F7EA55F74F918333
:103F4000808382829382A482B582C682D7820E94B5
:103F50005A4D90939F0880939E0880910702811587
:103F600051F1809171008260809371008091900086
:103F70008068809390008091A308811521F080E0F3
:103F80003FDD0E94E2091092070215C0E80133E00C
:103F9000CC0FDD1F3A95E1F7CA55D74FA501940123
:103FA0006A817B818C819D810E94A65E81111EC0E9
:103FB0000E151F052CF0CDB7DEB7EDE00C94345F85
:103FC0000F5F1F4F88E0FE013896DE0101900D92D1
:103FD0008A95E1F70E945A4D998788878A869B8641
:103FE000AC86BD86CE86DF862896E2CF01501109C9
:103FF00080CFC093A50892CF0F93CF93C82F809105
:10400000D00D811509F18C2F8554990BBC01072E19
:10401000000C880B990B0E945A5E20E030E040E4CF
:1040200051E40E94F05D9B01AC0160E070E080E033
:1040300090E40E94C75B20E030E04CED53E40E9426
:10404000285D4FEF5FEF2EDF8091CF0D811569F076
:104050002C2F2F77E0914B0AF0914C0A0FE740E9A3
:1040600063E070E08BE49AE00995CF910F91089599
:104070006330710509F048C0842F807F803821F1BA
:10408000803909F041C0622F6F776953770B072E93
:10409000000C880B990B0E945A5E20E030E040E44F
:1040A00051E40E94F05D9B01AC0160E070E080E0B3
:1040B00090E40E94C75B20E030E04CED53E40E94A6
:1040C000285D4FEF5FEFEECE622F6F776953770B6E
:1040D000072E000C880B990B0E945A5E20E030E0FE
:1040E00040E451E40E94F05D9B01AC0160E070E0AF
:1040F00080E090E40E94C75B20E030E04CED53E4A8
:104100000E94285D0C949B144C3F11F40C943614BF
:1041100008951F920F920FB60F9211240BB60F92B3
:104120007F928F929F92AF92BF92CF92DF92EF9247
:10413000FF920F931F932F933F934F935F936F9330
:104140007F938F939F93AF93BF93CF93DF93EF931F
:10415000FF938091940890919508A0919608B09152
:1041600097080196A11DB11D80939408909395081E
:10417000A0939608B0939708609194087091950861
:1041800080919608909197080E94585E8B01D82FD5
:10419000C92F20E030E040E85CE36091980870911E
:1041A000990880919A0890919B080E94285D9B0134
:1041B000AC01B8018D2F9C2F0E94A65E81150CF4D6
:1041C00051C110929408109295081092960810927E
:1041D00097087090A4088091A308811103C07114FE
:1041E00009F49CC00E945A4D7C01711020C0712CB2
:1041F0008091A308C72D811589F0C0919C08C11139
:1042000003C0C0919D08C72906EA18E0E12CF12CF3
:104210008091A508E816F1040CF4E9C08091A0088B
:10422000811509F47CC01092A008C82F78C0C091F5
:10423000F808D091F9080E945A4D0091A1081091F8
:10424000A2088C1B9D0B8017910788F20E945A4D83
:10425000C00FD11F8C010C1B1D0BE092F808F092CF
:10426000F9088090920890909308E4012196D093E9
:104270009308C09392080E945A4D90939F08809390
:104280009E08C0909008D0909108CC15DD0558F09C
:1042900080918F08811509F43FC010929308109205
:1042A0009208C0E0D0E0E0908C08F0908D088091FA
:1042B0008E085E0163E0AA0CBB1C6A95E1F78111D0
:1042C0003BC0F40153E0EE0FFF1F5A95E1F7EE0DEE
:1042D000FF1DD701AA0DBB1D2D913D914D915C9104
:1042E00060817181828193810E94A65E811124C0C8
:1042F00081E080938E084FE050E060E070E0CB01F9
:10430000D1DD90929308809292080FE010E0109314
:10431000A2080093A1086CCF0E943614C0E08091DF
:10432000A308811183C08091A40881117FC00E94DD
:10433000410A0E944C0A96C010928E08F701EA0DBD
:10434000FB1D64817581868197810E94AF5E9B0110
:10435000A3E5B7E00E94B86020EF30E040E050E015
:104360000E94966081E0C81AD10840EF842E912CFB
:10437000A12CB12C2017310718F4CC15DD05C8F09D
:10438000D0939308C09392080217130768F5F901B8
:10439000E01BF10B8F0183E0CC0FDD1F8A95E1F765
:1043A000CE0DDF1D688179818A819B81A8017ADD2C
:1043B000AECF021B130B2196FE0193E0EE0FFF1F01
:1043C0009A95E1F7EE0DFF1D6481758186819781D5
:1043D0000E94AF5E9B01A3E5B7E00E94B860A50113
:1043E00094010E949660C6CF01E010E0D4CFF8019E
:1043F000C680D780C60101978E3F9F4F88F4F80191
:10440000A080B1800E945A4D8A199B098C159D0588
:1044100038F0F80162817381848195810E949B1438
:10442000FFEFEF1AFF0A085F1F4FF2CEC115D1F060
:1044300080E0E6DA0E94E2098091A508823008F463
:1044400078CF81E0DDDA8B01D82FC92F20E030E072
:10445000A9010E94A65E811125C0809180008F7302
:1044600080938000FF91EF91DF91CF91BF91AF9149
:104470009F918F917F916F915F914F913F912F917C
:104480001F910F91FF90EF90DF90CF90BF90AF9072
:104490009F908F907F900F900BBE0F900FBE0F904C
:1044A0001F9018958091800080688093800020E0A4
:1044B00030E040E051E4B8018D2F9C2F0E94285D30
:1044C0009B01AC0160E074E284E79BE40E94F05D34
:1044D0008B01D82FC92F0E94AF5E462F572F5093C4
:1044E0008700409386006091060270E080E090E0D3
:1044F0000E945A5E98014D2F5C2F0E94285D20E09B
:1045000030E048EC52E40E94F05D0E94AF5E462F1E
:10451000572F5093890040938800A4CFA6E0B0E0C5
:10452000E4E9F2E20C94235F9093E30B8093E20BB7
:10453000811520E2920728F405D82696E2E00C9433
:104540003F5F80EF89838A830E945A4D8160BC015E
:1045500049815A8181E090E00E94CF37EECFCF931E
:10456000DF93D82FC92F0E94504B80915813909100
:1045700059130E9439138D2F9C2FD0DFDF91CF91DB
:104580000895ABE2B0E0E7ECF2E20C94135F7C013B
:10459000DC0114968C91811509F475C160E0C701A6
:1045A0000E94B30D9C01F7018681803170F4409127
:1045B0008B0C90918A0C491333C09091860C911505
:1045C00021F09091870C903158F1D70115969C916C
:1045D000911110C02115B0E53B0708F086C02115E8
:1045E000E0E23E0708F096C0283E310590F4203EF8
:1045F0003105B0F43093800C20937F0CD7011296D4
:104600008D919C9190937E0C80937D0C10927A02F8
:1046100007C0C9019A9581159F4160F72111EACF22
:1046200061E0C7010E94B30D8C01F70185818115FE
:1046300029F18091C2119091C3110097F9F00817E8
:104640001907E1F0FC01FF27807E9927892B09F0EB
:1046500063C044E0EE0FFF1F4A95E1F7EE53F04FC1
:1046600085818460858311830083CF0163D9109293
:10467000DD1161E0C7010E94B30D8C018091AB0D8B
:10468000811151C0D70115968C91811509F4B0C0E4
:104690000115B0E51B0708F096C00115E0E21E0702
:1046A00008F0F5C00115F7E01F07E9F1C0F5C801F2
:1046B000805E91090897B8F13091DA118091DD118F
:1046C0002091D81199E0F701A7E9BDE001900D9282
:1046D0009A95E1F710939F0D00939E0D1092A10DF6
:1046E000832B822B8093960D1EC0203E42E534071B
:1046F00060F4203852E5350708F092CFC9018052A6
:104700009245809708F076CF8BCFC90187579C4799
:104710000297F8CF8031F6CFE0E0F0E0A1CF0115AD
:104720003FE0130749F6F70185818111ADC10115FD
:1047300027E5120708F4D6C2011538E5130708F07B
:10474000A0C2680147E5D41A6CEA7DE08C2D0E9476
:104750005418892B31F5C601B4E0880F991FBA951A
:10476000E1F7FC01EE53F04F2281213009F074C2D1
:104770002091AC0D3091AD0D232B99F02091AE0D11
:104780003091AF0D232B69F02091B00D3091B10D18
:104790004091B20D5091B30D242B352B232B09F4EE
:1047A00065C20539F4E71F0709F08FC2D7011596D6
:1047B0008C91811511F40C945A318091B70D90E0D1
:1047C00008960C948E31003E42E5140750F40036F2
:1047D00052E5150708F0A7CFC8019255803491051E
:1047E0006ACF980127573C472530310508F064CF40
:1047F0000937BCE71B0709F04FC020919E0D30918F
:104800009F0D232B79F18115A1F081E00E94F70C17
:104810008091960D0E94891989E0E7E9FDE0ADE8F5
:10482000BCE001900D928A95E1F78091A10D8093F3
:104830008C0C86E0F701ADE8BCE001900D928A9502
:10484000E1F780918C0C8093AB0D8DE89CE099DEB4
:104850001092AB0DF7018581811104C08091960DF6
:104860000E9497198091DE118770811561F0D70140
:1048700015968C91811539F08091631382FF03C0E6
:1048800082E00E943706AB96E2E10C942F5FD701DD
:1048900016968C9180310FCF0A37FCE71F0709F07D
:1048A00042CF811509F4C5C0A0909E0DB0909F0D18
:1048B0002091960D2CA32983BE016F5F7F4FC50108
:1048C0000E94BD0B2C0139813AA736E9C32E3CE08A
:1048D000D32E01E010E022242A94D60117963C90B2
:1048E000179733FE53C06D907C90119712968D9060
:1048F0009C90139746145704B9F41496BC91B8A72A
:10490000232DF60146816B2F8AA50E94D70B8115B6
:1049100059F088A50E944505281634F4D60115964D
:104920009C918401192B282E48145904C9F431FE96
:1049300017C0F601F581F8A7232DD60116964C91E4
:104940006F2F8AA50E94D70B811551F088A50E9470
:10495000450528162CF4F60194818301192B282E85
:1049600030FE14C0FFEF2F1211C00130110571F499
:10497000232DD60116964C9160E08AA50E94D70B94
:10498000811521F0F60185818401182BF8E0CF0E06
:10499000D11C26E93DE02C153D0509F09ECF0130E4
:1049A0001105E1F58CA182958F703CA1832B8F704E
:1049B00011E0303108F410E01295107F182BA1148B
:1049C00040E2B40620F5A11451E0B50608F055C048
:1049D0000A2D812F8D704A2D811509F451C06AE08E
:1049E00086E097E00E94080D282F30E02115310560
:1049F00051F4402F66E188EE96E00E94080D282FC2
:104A000030E0811549F0F901F12B8F0107C0C50194
:104A100090528115904390F100E010E087E0E2EAC7
:104A2000FDE0DF011D928A95E9F71093AA0D00932E
:104A3000A90D8091A90D9091AA0D892B09F412CF8F
:104A4000F7018581811539F08FEF0E94F70C809175
:104A5000A10D8093A00D86E0F701A2EABDE00190D0
:104A60000D928A95E1F78091A00D8093AB0D82EABB
:104A70009DE087DD1092AB0DF5CE1B29BB24A8CF9E
:104A800068E08EEF96E0AECF9801375720383105B9
:104A900008F0F7C0003108F0E5CE6EE278E080E083
:104AA00090E00E94060F8111DDCE812C912C5401E3
:104AB000011147C004E0AE014F5F5F4F6A01D601AC
:104AC000E02F1D92EA95E9F724013501FFEF4F1A17
:104AD0005F0A6F0A7F0AC501B4010E94060F89832D
:104AE000811509F4BFCE813009F0B2C0A50194014F
:104AF0002E5F3F4F4F4F5F4F2CA33DA34EA35FA3AD
:104B0000C301B2010E94060F182F8A83811509F490
:104B1000A9CE8FEF810F833070F56CA17DA18EA19E
:104B20009FA10E94060F8B83811519F0C6010E9478
:104B3000B7562401350133E0430E511C611C711C32
:104B400049C0FFE28F16F8E09F06A104B10409F402
:104B500089CEC501B4010E94060F2FEF821A920A76
:104B6000A20AB20A8111EDCF0150A2CF4CA05DA0E4
:104B70006EA07FA02FC08BEF810F833098F52401AA
:104B8000350143E0440E511C611C711C6CA17DA1D8
:104B90008EA19FA10E94060F8B838115D9F0C301BE
:104BA000B2010E94060F8C83811569F08B819C8174
:104BB00081305FEF950710F0982F8827163069F045
:104BC000173071F0CCDC2401350154E0450E511C46
:104BD000611C711C5301420172CF0E94504BF3CFF4
:104BE0009DDCF1CF143009F0C1CF6CA17DA18EA165
:104BF0009FA10E94060F182F2401350184E0480E62
:104C0000511C611C711CC501B4016D5F7F4F8F4F3A
:104C10009F4F0E94060F111509F424CE811509F447
:104C200021CE8150990B4FEF489F9001499F300D45
:104C30001124A12FA150BB0B2A0F3B1F215031097A
:104C400048F2EFE9FFE03197F1F700C00000F6CF3E
:104C5000C6010E94B756BECF223009F0A2CD2091E6
:104C6000B00D3091B10D232B09F49BCDFC01E9531C
:104C7000F04F20812E7F20838E53904F0E949A1CEC
:104C800090CD003854E7150739F4811511F40C94D0
:104C90005A310E94FE0DE6CD013894E7190711F054
:104CA0000C947A31811511F40C945A310E944C15F0
:104CB000D9CDD70115968C91811511F40C945A31E8
:104CC0008091B60D80FDF2CFE4CF0039B4E71B0729
:104CD00049F4F7018581811511F40C945A310E9431
:104CE0000D0EC0CD0139F4E71F0751F4D701159619
:104CF0008C91811511F40C945A310E94B518B2CDE3
:104D00000239B4E71B0759F4F7018581811511F4C5
:104D10000C945A318091D00D8111EFCFE0CF011565
:104D2000F1E71F0751F4D70115968C91811511F405
:104D30000C945A310E94160E95CD0130B1E71B0735
:104D400049F4F7018581811511F40C945A310E94C0
:104D5000741588CD0230F1E71F0761F4D70115966D
:104D60008C91811511F40C945A318091CF0D8111E1
:104D7000EECFE0CF0339B4E71B0711F00C945A31A2
:104D8000F7018581811511F40C945A310E94AC18F9
:104D900020913B0330E02F5F3F4F23703327209358
:104DA0003B0348E2429FC001439F900D112465E000
:104DB00070E085569D4F0C949831D70115964C9113
:104DC000411509F44AC0003E110561F40E94AC1877
:104DD00081E08093CE0D1092CD0D1092CC0D1092EB
:104DE000CB0D40CD023E110571F40E94AC188091AC
:104DF000CE0D811519F081E08093CD0D1092CE0D6E
:104E00001092CC0D2FCD033E110591F48091CD0D64
:104E1000811519F10E94AC181092CE0D81E080939B
:104E2000CC0D1092CA0D1092C90D1092C80D1ACD5A
:104E300080913C0390913D030A970235110541F0A2
:104E40000135110551F480913C0390913D030A9680
:104E500090933D0380933C0305CD80913B038111EA
:104E60000EC0F701218184E090E0821B91099081BE
:104E7000905FD92EFCE08F9FD00C112412C081309E
:104E800049F5D70111968C91119724E030E0281B49
:104E90003109822F880F880F820F9C919D5CD82E3C
:104EA000D90E8D2D411509F443C0A6D88091CE0DA1
:104EB000811551F08091CB0DE82FF0E0E854F24FCE
:104EC000D0828F5F8093CB0D0F3F110510F00C94B3
:104ED0006431C8CC823059F4F701218184E090E03C
:104EE000821B910990819D5CD92EF7E0C4CFFCE034
:104EF000DF2E8330B1F683E2ECEBF3E0DE011196B6
:104F000001900D928A95E1F7D7018C91FE01E80F8F
:104F1000F11D11968C9124E030E0281B3109808529
:104F2000BCE02B9F800D1124A9E0DA2ED80EB9CF5A
:104F30000E941215C9CF1092DA110E9460060E94D9
:104F40005A4D88579C4E9093D30D8093D20D81E09B
:104F50008093D10D87CC023AF2E51F07B9F158F4DE
:104F6000C80190528115904218F1013E110571F16E
:104F7000053E110503C0023B42E5140709F03FC09E
:104F800025EE30E02770332781E090E001C0880FE4
:104F90002A95EAF72091D40D3091D10D3115F1F019
:104FA000F70135813115A9F0282B2093D40D5ACC67
:104FB000D70116968C91803110F5812F99278F712A
:104FC00099278230910511F04297D8CF21EE30E039
:104FD000D9CF809582238093D40D44CC322F3823AF
:104FE000311569F0982F909592239093D40D0E94DB
:104FF000B113D70115968C91811509F433CC8091AA
:10500000D10D811509F47AC0C090DA11D090D81171
:105010000E945A4D88579C4E9093D30D8093D20D89
:10502000F7018581811509F469C08D2D8C298D7951
:1050300081118DC00115F0E51F07E0F5011520E491
:10504000120708F08BC0063E110509F457C0C801CD
:1050500090528115904208F042C0D70116968C916B
:10506000803108F46EC06801DD2480913F0380FF29
:1050700081C08DEF0E945806BDE2CB16D104A1F08D
:1050800008F08BC0F8E2CF16D10408F075C02EE10D
:10509000C216D10408F074C034E0C31AD1084AE142
:1050A000C416D10408F053C08091DD118260809352
:1050B000DD1166C0003EB2E51B07C0F4003CE2E52E
:1050C0001E07E0F4003AF2E51F0758F4003622E527
:1050D0001207A0F4C80192558034910578F0680158
:1050E000C4CF043B32E5130749F0F9CF09374CE749
:1050F000140718F507375CE7150788F3D7011596ED
:105100003C90311409F456C00E35BCE71B0709F476
:105110004DC00F35ECE71E0751F00D35FCE71F07BA
:1051200009F048C080913E03811509F43FC01092F8
:105130003E0380E00E94D55795CB0B378CE71807CC
:10514000D3CF812F8F718431C9F2863171F00E94E3
:105150009D198091D40D0E945206D0CFD70116968A
:105160008C91803108F07FCFC9CF76EEC72E72E1E7
:10517000D72E7BCF8FEF7ECF5AE2C516D10439F7F9
:105180008091D40D811531F08091DD1192E0892755
:105190008093DD110E942F19B1CF8CE4C816D10481
:1051A00079F39DE2C91692E0D906E9CF81E08093B8
:1051B0003E0358CB80913E03811149C0C8019755E9
:1051C0008115914008F0DFC05801F0EEAF22BB24FA
:1051D000A114B10409F046CBF801FF2754E0EE0F0B
:1051E000FF1F5A95E1F79F012E53304F6901D701F8
:1051F00015968C91E953F04F908180FB90F9908344
:10520000811509F4FBC10E945A4D9093C5118093FA
:10521000C411F60182818F5F82838091DD119091AC
:10522000DA11892B83838091D81184834681578139
:1052300066857785C6010E941D0DD60115968C9155
:1052400081FF5801B092C311A092C2119CC03801D5
:1052500030EE631A71085090D9118091DA11582AF2
:105260008091D811582A48E06416710408F05EC095
:1052700098012770332781E090E001C0880F2A95BC
:10528000EAF7311409F44FC0582AD7018D919C9147
:105290000E947D1321E030E0F90102C0EE0FFF1FF4
:1052A0008A95E2F7FDA3ECA32091B80F3091B90FD6
:1052B0003BA72AA74091C00F5091C10F59A748A7FB
:1052C00067EDC62E6DE0D62EA12CB12C511005C075
:1052D000D60112968C9181111BC0F601838190E05A
:1052E0002CA13DA182239323892B91F08085982FB7
:1052F0009770911101C087E038E06316710408F0DF
:10530000A8C0311409F4A1C0869581708111A6C08E
:105310009FEFA91AB90AAFE0CA0ED11CB0E2AB16D2
:10532000B104A1F61CC080955822AFCF31107AC0CD
:105330008091C00F9091C10F0817190781F4109246
:10534000C10F1092C00F1092BC0F1092BD0F10929F
:10535000BE0F1092BF0F1092BB0F1092BA0F809128
:10536000B80F9091B90F009709F428CFE8E06E16B6
:10537000710408F02DC1652D0E94AF0C811103C08E
:1053800081E00E94D5578091551380FFA7C10E94EC
:105390005A4D5C01F7018581811509F4B1C18091F5
:1053A0003F0382FF06C040E0B50180E090E00E942C
:1053B00043580431FCE71F0709F49EC105312CE76F
:1053C000120709F438C103313CE7130709F479C126
:1053D000C80190528115904308F037C11092C9114D
:1053E0001092C811F7019581911509F4B7C7109271
:1053F000D311980130572332310508F09DC784E05E
:1054000090E00E9421609093631380936213F801EF
:10541000E150F047E232F10508F039C2ED5EFE4995
:105420000C945D5F1093C10F0093C00F0E946F4DED
:105430006093BC0F7093BD0F8093BE0F9093BF0F0E
:105440001092BB0F1092BA0F20CF82FB882780F9F1
:105450005DCF311409F45CCF80FF5ACFD6018D9017
:105460009C900815190519F4311409F451CFEAA5D7
:10547000FBA5EC15FD0509F44BCFD6011D96ED916A
:10548000FC91309721F08081811509F441CF652D81
:10549000C6010E94AF0C811509F43ACF81E00815CE
:1054A000190509F080E0482E43208114910441F051
:1054B000411006C0E8A5F9A58E169F0609F028CF71
:1054C00080E00E94D557D092B90FC092B80F81E00A
:1054D0008093B70F8FE08A9DF0018B9DF00D112412
:1054E000E952F24F85818093D60D41100EC0811490
:1054F000910459F0808191819C0124503109213A15
:10550000310508F049C00E940B4D8FE08A9DF001E3
:105510008B9DF00D1124E952F24FC680D780C60151
:105520009A9581159F4110F420EED22299249394EC
:10553000C60101978F339E4708F0912C8FE08A9D1A
:10554000D0018B9DB00D1124A952B24F1996ED9147
:10555000FC911A97309731F01B966D917C9181E008
:10556000099598229114A9F08FE08A9DF0018B9DF6
:10557000F00D1124E952F24F868197810E941205A5
:105580008093D50DC60148E06416710440F40E9472
:1055900069180E942F190AC00E945B1AB6CF04979F
:1055A000813A910548F48C2D0E94720D411409F442
:1055B00005CE0E942F1956C90E942F198FE39CE92E
:1055C0000197F1F700C000008C2D0E94A619EECFC4
:1055D000DC012D913C910217130741F4311009C0F1
:1055E0001092B70F80E00E94D557E8CD311409F42E
:1055F000E5CDFC01808585FDE1CDF4CFF901448541
:10560000558566857785C9010E941D0DD6011596C1
:105610008C9181FFB8CEC6010E94821C8091C2117C
:105620009091C3110817190709F0ADCE1092C3115C
:105630001092C211A8CE90913F03892F8E7F90FFC8
:10564000816080933F030E94611C80913F0380FF33
:1056500045C00832110508F069C00E31110508F087
:1056600076C0C80104974A9788F58091551384FD48
:105670002DC0D70115968C91811509F4D6C0809163
:10568000D8119091DA11892B8D7F811509F464C0AE
:105690001092C9111092C8118091551381FD5CC000
:1056A00060E0C8010E942E1860E0C8010E943458D2
:1056B0008091D8118D7F0E94EC1C82E00E943706F9
:1056C000D1C880913F03816080933F03F7018581BA
:1056D000811521F01092C9111092C811D7011596A9
:1056E0008C91F801E851FC47E730F10508F07ACEDB
:1056F000EB5CFE490C945D5F80913F038E7FA1CFF0
:1057000080913F038F7E013E110531F0053E11056A
:1057100031F480913F038F7D80933F0396CFC80182
:1057200090528115904308F090CF5CCE093311055B
:1057300058F40D32110518F40B32110539F6809129
:10574000551382FDC3CF95CF04361105F7CF809155
:10575000551383FDBBCF8DCF89E0F701AAECB1E1F2
:1057600001900D928A95E1F71092CD111092CC1113
:105770008091C8119091C91108171907C9F5209196
:10578000551325FF35C030913F0331FF02C026FF7E
:105790002FC02091C6113091C7116501C21AD30ADA
:1057A0000E94D258C816D90618F58091DA1181FFE7
:1057B00008C080913F03806180933F0382E00E9494
:1057C000B1138091DA1185FF08C080913F03806298
:1057D00080933F0380E20E94B11360913F0366957E
:1057E00061708091C8119091C9110E9434583AC8D3
:1057F0008091D811D090DA11D82AD1FADD24D0F8CE
:105800008D7F0E94EC1C1093C9110093C811B092B7
:10581000C711A092C611DD0C6894D2F890913F0395
:10582000997FD92AD0923F0348CF40E0B501C80103
:105830000E94435817C806E221EE41EE6AE17CE778
:105840000E94EE580FC807E225EE45EE6BE17CE7BB
:10585000F7CF06E221EE40EE68E17CE7F1CF07E208
:1058600025EE44EE69E17CE7EBCF06E221EE42EE65
:105870006CE17CE7E5CF07E225EE46EE6DE17CE7E3
:10588000DFCF08E221E045EE6EE17CE7D9CF8091E1
:10589000621381608093621382E693E10E94BF0DE0
:1058A0000E94D81A0C9432248091631388608093EC
:1058B0006313F2CF809162138260ECCF8091621308
:1058C0008460E8CF809162138860E4CF8091631395
:1058D0008160EDCF809163138260E9CF8091621384
:1058E0008061D8CF809162138062D4CF809162139F
:1058F0008064D0CF0E94D81A809162138068CACF8A
:10590000809162138C608093621364E070E080E8A1
:1059100093E00E946057C0CF8091631383608093AF
:10592000631364E070E080E693E0F3CF809162134C
:105930008E7FB0CF80916313877FB9CF8091621340
:105940008D7FA8CF809162138B7FA4CF809162134B
:10595000877FA0CF809163138E7FA9CF809163133F
:105960008D7FA5CF809162138F7E94CF809162133B
:105970008F7D90CF809162138F7B8CCF0E94D81A3D
:10598000809162138F7786CF80916213837F80939B
:10599000621362E070E080E593E0BBCF8091631317
:1059A0008C7F8093631362E070E080E493E0B1CF7A
:1059B00080916213992782FF939590FB82F990FB67
:1059C00083F98093621383FFE4CF9FCF80916313A9
:1059D000982F909590FB80F990FB81F98093631349
:1059E00081FFE1CF9ECF90916213892F8F7B96FF2D
:1059F000806450CF0E94D81A90916213892F97FB30
:105A000087F9805847CF61E08EE090E00E943560D2
:105A100043CF60E0F9CF90916213892F8F7E94FF7E
:105A2000806138CF90916213892F8E7F90FF8160C3
:105A300031CF90916313892F877F93FF886037CF91
:105A400020E09DC48091D411811521F085E30E944E
:105A50000B4DAFCD89E2FBCF0E94E00A0C943224BB
:105A60008115A9F10E942A0B0C9432248115A9F109
:105A70000E944B0B0C9432248115A9F10E94600BFB
:105A80000C9432248115A9F10E94780B0C943224D5
:105A90008115A9F10E948E0B0C9432248091DA11A9
:105AA0008272F801E054F847ED30F10560F5E45CEE
:105AB000FE490C945D5F0E94EA0A81E00E94D80AC8
:105AC0000C9432240E94F80AF8CF811559F20E94F2
:105AD000200B0C943224811559F20E94420B0C9435
:105AE0003224811559F20E94540B0C9432248115F2
:105AF00059F20E946C0B0C943224811559F20E94C9
:105B0000840B0C9432240737FCE71F0701F1083798
:105B10002CE7120741F19801205E32452032310511
:105B200038F5911125C00F7181E090E0AC0102C001
:105B3000440F551F0A95E2F78A01642F83E090E035
:105B40000E943560802F0E947F050C94322481E0F2
:105B5000911559F00E94850543E062E081E00E94C2
:105B60009D050C94322482E0F3CF0E948F05F4CF80
:105B70004091D51180913913282F30E02095309530
:105B800070E024233723232B19F048234093D511A9
:105B90000B375CE7150751F4911511F40C9432247E
:105BA0000E9448050E94D00C0C943224003482E5F7
:105BB000180708F04EC00032A2E51A0708F050C0DE
:105BC0000115B0E51B0720F50115E0E41E0708F0FC
:105BD0005EC0911509F475C00A35BCE71B0709F4CE
:105BE000F1C008F0D5C00130FCE71F0709F4E8C098
:105BF00003302CE7120709F4DDC001153CE7130759
:105C000009F05FC00E941A5A0E949F4D0C943224E2
:105C10009801305521153240E0F6980145E036955F
:105C200027954A95E1F7822F8F702091D51130E0AA
:105C300041E050E0082E02C0440F551F0A94E2F7DD
:105C400024233523232B29F29111ACCF1092DA11A2
:105C5000B0CC9801205C32452032310508F0B9CF34
:105C6000802F8F712091D51130E041E050E0082E57
:105C700002C0440F551F0A94E2F724233523232B37
:105C800009F4A7CF911511F40C9432248BCFD701CE
:105C900016968C91803108F09CCF911112C0212F63
:105CA0002F7081E090E002C0880F991F2A95E2F7DB
:105CB0002091D51130E082239323892B11F00C948D
:105CC0003224F70187819085009709F47FC00E94F4
:105CD0005E07082FD92E86E0F701DE0111960190AC
:105CE0000D928A95E1F7F701B580C680C2949FE0D6
:105CF000C9228091DE118770811501F19B2CB114AE
:105D0000F1F08D2D807F803461F080E2800F88304B
:105D1000A8F08D2D807E803221F4023078F0C114FD
:105D200069F08091631382FF09C082E00E94370608
:105D30008091DE118770992493948111912CAD2C60
:105D4000A2948FE0A822F8E0AF1609F480C129E000
:105D5000A21608F08AC034E0A31608F04EC01D2D2C
:105D60001F7042E0A41608F493C08D2D807F80320E
:105D700011F01295107F011509F4BEC0013009F42D
:105D800028C1B11409F434C1C11409F4CFC094C0BE
:105D90000B354CE71407C1F080916313002482FF98
:105DA0000394802D0C355CE7150709F08ACF0E941B
:105DB000C60D87CF6FEF7FEF80E090E00E944F60CD
:105DC0000E94A60D81E0F3CF80E0F1CF8581C080F5
:105DD000D180811569F0C6010E94D413182F682F55
:105DE000C6010E944713B601812F0E94B9136FCFDD
:105DF000C6010E947D13182FF6CF54E0A51609F4B2
:105E000009C1AA2DA850BB0B149718F40E94BE1804
:105E1000912C802F9D2D0E945B05811541F0B114BE
:105E200009F41DC2C11409F411C210926613911431
:105E3000B1F08091DE1180FD12C0D70115961C9241
:105E40008695869586950E948505C7010E94C12288
:105E50008091DE118695869586950E948F0560E07B
:105E6000C7010E94B30D0C94432489E0A81609F4DD
:105E70005EC186E08A0D8F70823018F6023F09F00D
:105E800066C18D2D8F71B1105FC10E948505B9CF9C
:105E900090E1D91610F01295107FB114B9F01115D8
:105EA00059F080E2800F883010F0011109C0812F75
:105EB0000E9452060E942F19802F0E94A619A1CF7E
:105EC0008091DD11812B8093DD11F4CF802F0E9412
:105ED0005B1A111509F495CF80E2800F883010F01D
:105EE000011104C0812F0E94B11303C0812F0E94B1
:105EF00058060E942F1985CF8091631382FD12C02E
:105F0000B11449F0111529F0812F0E9452060E9408
:105F10002F1980E0D2CF80E00E945B1A111509F49E
:105F200070CFE0CFB11491F1C11004C0812F0E9455
:105F3000831967CFB1E0CB1211C08090D811812FA7
:105F40008821181709F45DCF0E945A4D9093D711FC
:105F50008093D611812A8092D81153CF8091561305
:105F6000823008F44ECFC8124CCF812F0E94831983
:105F7000812F0E94D61C8091D911912F9823191737
:105F800009F43FCF812B8093D9113BCFC11012C0B0
:105F9000812F0E949219812F0E94D61C8091D911C5
:105FA000912F9823911509F42CCF10951823109355
:105FB000D91127CF80915613823008F422CFE1E027
:105FC000CE121FCF8091DA118123811509F419CFE8
:105FD000DFCF80915C13B11421F08C1508F411CF40
:105FE000A5CFC81608F00DCF812F0E94921909CFB6
:105FF000C114D1F380915A1390915B13093321F0AE
:1060000080915813909159130E943913802F0E9448
:106010005B1AF7CE8D2D869586958370811569F074
:10602000813009F0EECE802F9D2D9370B11002C00B
:1060300080E090E00E944A0DE4CE802F9D2D937069
:10604000B11002C080E090E00E94220DDACE8D2DCA
:106050008370811133C0B110D4CE402F4295469544
:106060004770440F440F802F8F70042E01C0880F9B
:106070000A94EAF7202F207104FF07C02FE030E0D8
:1060800001C0220F4A95EAF720953D2D36953695A9
:106090003370323071F0333051F040913813313079
:1060A00029F0822B84230E947F05ABCE842B822B88
:1060B000FACF822B909138138927F5CFB11459F17B
:1060C000D0FE9FCE402F429546954770440F440F17
:1060D000802F8F70042E01C0880F0A94EAF7202FBA
:1060E000207104FF07C02FE030E001C0220F4A9565
:1060F000EAF720953D2D369536953370323091F084
:10610000333071F040913913313049F0822B8423C0
:106110000E94820576CE823008F473CED3CF842BD2
:10612000822BF6CF822B909139138927F1CF1D2D29
:106130001F70B11429F0812F0E948505802FF7CEA2
:10614000802F0E949219812F0E948F055ACE60F4F1
:10615000003FB9F0013F81F0B11409F472C0C110E1
:10616000ABCE8D2D8F7191CE033FF9F0043FA1F797
:106170008091631382FD25C08D2D8F71B11421F3A1
:1061800084CE80915C13B11461F0C81608F039CE4A
:106190002D2D2F7181E090E001C0880F2A95EAF73C
:1061A000C2CF8C1508F42DCEF3CF80E0B11409F4E2
:1061B000AFCF81E09D2D9F7101C0880F9A95EAF7BE
:1061C000A7CF80915613823048F1B114C9F0909155
:1061D000DE119770943059F41092DE111092E01194
:1061E0001092DF118D2D8F710E948F050FCE63E00D
:1061F000C81608F00BCE8D2D8F710E94BF1C06CEE5
:10620000C81640F01092DE111092E0111092DF11CA
:1062100064E0F1CF81E00E943706F8CDB11431F08F
:1062200063E08D2D8F710E94BF1CEBCD81E00E9439
:106230003706F2E0CF1608F4E4CD82E00E9437067C
:10624000E0CDC110D7CE8D2D8F717ECF8091DC1126
:106250008093DB118091DA118093DC11E8CD40E06E
:1062600060E089819A810E943D5A9C011091DA1167
:10627000C11429F0109266131093DC11D8CD8091CF
:1062800064139091651328173907B1F7809157135C
:1062900082FFF0CF80916613811561F38091DB114D
:1062A0000E948319802F0E94CD1A8091DB110E94D9
:1062B0009219E0CF8091D00D81110C94DD26809150
:1062C000CF0D81110C94DD260337FCE71F0711F079
:1062D0000C94AB27F7018581811511F40C943224BD
:1062E0008091D10D811511F40C949B270E949D196A
:1062F0000C9432240238B4E71B0711F40C9459268D
:106300000439B4E71B0711F00C94D123F701858100
:10631000811581F28091B70D90E0019669E070E0FF
:106320000E944A5F8093B70D64E070E08BE792E0D3
:106330000E9460570C9432240631FCE71F0799F045
:106340008091DA118272F801E052F847EB30F105E2
:1063500008F0D9CBE75BFE490C945D5F06312CE772
:10636000120709F09BCB8091DA113091541330FF62
:1063700004C0282F2474211163CB282F2A7A31FFDF
:1063800004C0482F4171411120E032FF04C0482F62
:106390004878411120E033FF03C08272811120E070
:1063A000911509F44FCB81E0211101C080E0809369
:1063B000D41185E3211101C089E20E94720DF9C850
:1063C000A0E0B0E0E6EEF1E30C941E5F8091870C54
:1063D000803108F049C08091860C811509F444C0D1
:1063E000C0918B0C89E0D82E80918A0C8C17E1F13A
:1063F000EC2EF12CDC9EE0011124FE01ED5DF34F4B
:1064000084818115B1F191818091820C981331C002
:1064100090818091810C98132CC08581811129C0B5
:10642000028113818091830C9091840C081B190BBD
:1064300060E081E89CE00E94B30D0E94D2580817EA
:106440001907B8F48091870C8F7080618093870C56
:10645000C75DD34F88818F708061888381E89CE01D
:106460000E94C1220E942D06CDB7DEB7E7E00C9452
:106470003A5FE7012196C770B7CFCF92DF92FF92C4
:106480000F931F93CF93DF93182F092F89E0F82ED6
:10649000C0918B0C80918A0CC81799F1FC9EE00189
:1064A0001124CE018D5D934F6C01FC018581811516
:1064B00089F0C6010E940B14811561F0FE01E75DB1
:1064C000F34F20812F7020612083F601808191811C
:1064D0000E94F81AC6010E94C12220918B0C30E064
:1064E0002F5F3F4F2770332720938B0CCD5DD34F09
:1064F00089818013CDCF88818113CACF8D81811589
:1065000039F2DF91CF911F910F91FF90DF90CF90E3
:106510000895EF92FF921F93CF93DF93EC012091A8
:106520007A02211541F010E0812FDF91CF911F9168
:10653000FF90EF900895EA80FB80E61AF70A24EFB7
:10654000E21621E0F20678F760E0CE010E94B30D7A
:106550009C0130522115304330F70E94F805811517
:1065600011F380917F0C9091800C0E94F805182FF8
:106570008115C9F28091601390916113853F21E0EC
:10658000920710F084EF91E0E816F90660F68E812C
:106590008F7080618E83888199810E94F81A0E9491
:1065A000BC05CE010E94C122BFCFAFE0B0E0EBED51
:1065B000F2E30C94145F8C0186E0F801DE011A9678
:1065C00001900D928A95E1F7D8014C9011963C907C
:1065D00011971296ED90FC90139714965C90149777
:1065E00015966C9061100CC05091220C252F30E054
:1065F000E0E08E2F0E2E000C990B821793073CF1D2
:1066000051E8A52E5CE0B52E8091850C811151C01A
:106610005114D1F0611409F43FC3C8010E940B1456
:10662000811509F439C360917D0C70917E0CC8010D
:1066300070DF811109C089E0F801A1E8BCE0019098
:106640000D928A95E1F7BCDEFF24F39497C0880F82
:10665000991F8E5E934FDC0111964C911197431157
:1066600003C08C91481611F0EF5FC3CFEF3F41F2AA
:10667000D80116968C9116978F70806116968C9320
:10668000E517A0F4AFEFA50FA093220CEA1770F462
:10669000F0E0EE0FFF1FEE5EF34FB0E0AA0FBB1F5E
:1066A000AE5EB34F8D919C91918380830E94BC0517
:1066B000A7CF60E081E89CE00E94B30D6C01709070
:1066C000860C8091830C9091840C4701881A990A5A
:1066D00060E081E89CE0711409F479C20E94B30D76
:1066E0000E94D2588816990608F026C2511409F45F
:1066F000ABCF8091820CF8019181B090870CF0E1D2
:10670000BF1608F0D3C198135BC09091810CD801DB
:106710008C91981355C02091880C3091890C179654
:106720008D919C912817390709F04AC0611048C023
:106730008B2D8F7080618093870C81E89CE00E9494
:10674000C1228091870CF8018683F090830CE09041
:10675000840C49E0D42E00918B0C80918A0C081790
:1067600051F0D09E800111240D5D134FD801159674
:106770008C91811108C00E942D06F12C8F2D2F962F
:10678000E1E10C94305FF801B280C380C8010E943F
:106790000B1481110EC0C8010E94C12280918B0C84
:1067A00090E001968770992780938B0CFB2CEC2C42
:1067B000D2CF6F2D7E2DC801ACDE8111EFCFDBCFA4
:1067C000F0E2DF1AC11420E3D20608F084C06110A1
:1067D00005C140E0632D842D0E94FB5981114FC0FB
:1067E00040E0632D842D0E94FB59F82E811509F499
:1067F00029C18091571380FFC0CF81E89CE00E949F
:10680000C12260E081E89CE00E94B30D8C01F09011
:106810008B0C7F2C98E0E92E21E8822E2CE0922E22
:1068200039E0432E80918A0C7816A1F0A72CB12C68
:10683000479CC0011124FC01ED5DF34F6F0160E046
:10684000CF010E94B30D582E692ED60115968C915A
:10685000811197C0B8E0EB1618F419E0EF10ACC046
:106860008A859B850ADE0E94BC050E942D0689E070
:10687000E1E8FCE0DF011D928A95E9F77ECF60E058
:10688000C8010E94B30D8091571383FFA9CFB801AF
:1068900081E89CE00E94C9058111A2CF8091870CFC
:1068A0008F7080618093870C8091810C9091820C15
:1068B0000E94F81A81E89CE00E94C122E1E8FCE015
:1068C00089E0DF011D928A95E9F78A859B85D5DDF0
:1068D0000E94BC0550CF611409F482CF8091870CCF
:1068E00081608093870C8091571381FF46CF81E8A8
:1068F0009CE00E94C12200918B0C80918A0C0817A9
:1069000009F4CCC0E02EF12CB9E00B9FC00111249A
:10691000FC01ED5DF34F6F01CF010E940B14811557
:1069200009F4BCC089E0F601A1E8BCE001900D9239
:106930008A95E1F7C701019687709927082F809300
:106940008B0C0E942D0689E0F82E80918A0C80170E
:1069500009F411CFF09E800111240D5D134FC80181
:106960000E940B14811107CFC8010E94C12280919F
:106970008B0C90E0019687709927082F80938B0CE1
:10698000E4CF10520115E0E31E0708F063CF8091B9
:10699000571383FD0AC0E72CC5010196F82FF77045
:1069A0007F2E052D162D46013DCFB601C4010E9454
:1069B000C905811589F3EFCF1F9DC00111248D5D9D
:1069C000934F0E94C12220918B0C30E02F5F3F4FEC
:1069D00027703327F22E20938B0C40CF8091870CA9
:1069E00081608093870C60E0C8010E94B30D8091A4
:1069F000571383FF78CFB80181E89CE00E94C90556
:106A0000811171CFF090870CE894F0F8F092870C28
:106A1000C8010E940B148111B0CE8F2D8F70806140
:106A20008093870C8091810C9091820C0E94F81ABF
:106A30000E94BC0581E89CE00E94C122E1E8FCE0E4
:106A400089E018CF8A859B850E94FE13292F229505
:106A50002F70903450F49F70223080F0911599F08F
:106A6000F8019681903178F489CE2A5F2F70223018
:106A700078F0C8010E94C122F72C80CE911519F040
:106A8000811509F47BCE805E883008F477CEF1CF93
:106A9000803F08F473CE815F8330F7CF89E0E1E86F
:106AA000FCE0DF011D928A95E9F74DCF98131EC0D7
:106AB0009091810CF8018081981318C02091880C66
:106AC0003091890C878190852817390779F46110F6
:106AD0000DC0B682C8010E94C12289E0F801A1E878
:106AE000BCE001900D928A95E1F7AECDC8010E94FD
:106AF0000B14811509F4D0C0611409F4CDC0809144
:106B0000870C803208F497CD8091810C9091820C93
:106B10009A838983FC82EB828091850C8D831E820F
:106B2000BF828091880C9091890C99878887CE01CB
:106B300001960E94C1227FCDD090870CF0E1DF1634
:106B400038F481E89CE00E94C12289E0D50193CE0F
:106B5000511409F479CD9091820CF8018181981338
:106B60001AC09091810C8081981315C02091880CD7
:106B70003091890C878190852817390761F461105D
:106B80000AC0D682C8010E94C12289E0D5011D92A7
:106B90008A95E9F759CDC8010E940B14811509F4B3
:106BA0007BC0611409F478C08091870C803208F4AE
:106BB00042CD8091810C9091820C9A838983FC82D2
:106BC000EB828091850C8D831E82DF82AACF0E948A
:106BD000B30D0E94D2588816990608F061C051146E
:106BE00009F432CD611409F457C09091820CF80178
:106BF0008181981339C09091810C8081981334C0A1
:106C00002091880C3091890C87819085281739074D
:106C100059F58091830C9091840CE81AF90A60E090
:106C200081E89CE00E94B30D80915E1390915F1308
:106C3000E816F90608F051CF8091870C80FD4DCF02
:106C4000803108F44ACFD80116968C931697982F66
:106C5000907F903F09F43ECF982F907F905F8F7088
:106C6000892B16968C9336CFC8010E940B14811580
:106C700071F060917D0C70917E0CC8014ADC811529
:106C800009F4D9CC89E0E1E8FCE0DF0180CF809114
:106C9000870C81608093870CC8010E94C122D4CCEC
:106CA00089E0F50111928A95E9F767CDA2E1B0E09C
:106CB000ECE5F6E30C94215F0A871B872C873D8760
:106CC0004E875F87688B798B8A8BCE010A966DDC45
:106CD000811128C020918A0C30918B0C89E0FE0133
:106CE0003A96DE01119601900D928A95E1F78E8514
:106CF0008115C1F0822F90E001968770992738178F
:106D00001906C1F199E0929FD0011124AD5DB34FF6
:106D1000FE01319601900D929A95E1F780938A0CCD
:106D20000E942D0619E080918B0C90918A0C891796
:106D300041F0189FC00111248D5D934F36DC811105
:106D400027C08E85811112C080917A0281110EC0F8
:106D50008C859D8520917D0C30917E0C821B930B40
:106D60008F3F9F4318F081E080937A026296E4E0BF
:106D70000C943D5F0E94D81A10928A0C10928B0CD2
:106D800089E0E1E8FCE0DF011D928A95E9F7CACFCE
:106D900080918B0C90E001968770992780938B0CE3
:106DA000C2CFEF92FF920F931F93CF93DF93809107
:106DB0003513E091C205CDE0811139C0CDB7DEB702
:106DC000E6E00C943B5FD1E0DE0FD093C205EE2EDF
:106DD000F12CCE9FF0011124E353FD4E84818115E7
:106DE00029F187819085892B21F4818592850196EF
:106DF00051F4008111812281338144815581668162
:106E00007781808553DFCE9DF001CF9DF00D112459
:106E1000E353FD4E14828091D10D811521F08091B4
:106E20003F0380FD0DC08FEF0E945806ED2F80912B
:106E30003513E81740F2109235131092C205BECFF9
:106E40008DEFF2CFA4E0B0E0E8E2F7E30C94145F3A
:106E50002091CC12298397E0992E01E010E02DE0DB
:106E6000322E34E0532E882483948091CB12998162
:106E7000891307C096DF0E94720C2496E1E10C94FE
:106E8000305F9981892F90E09C838B83FC01EE0F0A
:106E9000FF1FEF53FD4E80819181989ED001999EF6
:106EA000B00D1124FD01EF51FE4EFA83E9832481D8
:106EB00021115BC060903513EDECF2E160E070E011
:106EC000712C661508F04FC0A384B484A981BA81DF
:106ED000CD90DC902FEF3FEF412C442D50E0760118
:106EE000E40CF11CE40CF11CD701ED90FC90E114D2
:106EF000F10439F0AE14BF0409F0A90143949A01DA
:106F0000ECCF2F3F3207D1F1D80102C0AA0FBB1F2F
:106F10002A95E2F77A2A9801042C02C0220F331F27
:106F20000A94E2F7A901415051097416150629F592
:106F3000369EF001379EF00D1124E353FD4E989ECE
:106F4000D001999EB00D1124AF51BE4E12962D91D5
:106F50003C91139730872783548210821182928745
:106F6000818715968C920E94830C8B819C8101965F
:106F70009A8389838370898378CF14826F5F7F4F70
:106F80003D969FCF10923713109236131092A003A4
:106F90008091CB128093CC120E94720C02CFACE194
:106FA000B0E0E5EDF7E30C94135F4B8B5C8B6D8BDE
:106FB0007E8B8F8B692F988F192F811509F474C0E0
:106FC00040E08B899C890E943D5A9C01111549F033
:106FD0001092661390936513809364131092DD11E1
:106FE0000AC080916413909165138217930719F476
:106FF00081E080936613188A198A1A8A86E0FE0156
:107000007396DE011A9601900D928A95E1F78091B0
:10701000631382FF21C080913C1390913D13892B13
:10702000D9F00E945A4D2091DF113091E011821B5E
:10703000930B20913C1330913D138217930738F046
:107040008091DE1182FD03C082E00E9437060E941B
:10705000D71881110E9460068E858115D1F061E0FC
:10706000CE010A960E94B30D61E0CE010A960E94FD
:10707000B30D61E0CE010A960E94B30D5C0180352C
:107080002CE79207A9F48F85811531F181E0809377
:10709000A0030A851B852C853D854E855F85688903
:1070A00079898A8903DED5C0911509F4A4CF96CFDA
:1070B00081353CE7930729F48F85811569F062DFFC
:1070C000E8CF82359C4741F48F85811529F0809166
:1070D000A0038111F4CFDACF41EEE42E41E1F42E8A
:1070E000712C812C912C22242394312C6F84D70174
:1070F0006D917C91CC24CA94DD24DA9480E0282F11
:1071000030E0FB01E80FF11DE80FF11D40815181D6
:107110004115510539F0A416B50609F096018F5FA7
:107120006901EDCFBFEFCB16DB0609F475C1F7019E
:1071300044815090A0034111512CD70115964C90D9
:10714000159716969C911697611409F407C151146E
:1071500009F404C10091501310915113411015C04E
:10716000F10102C0EE0FFF1FCA94E2F76F019E2BE0
:1071700016969C932091C9123091CA12201731079C
:1071800020F41093CA120093C912910102C0220F79
:10719000331F8A95E2F7C9010197D70116962C9102
:1071A0002817190609F0BDC0C0903613D0903713C8
:1071B000C114D10409F451C00E945A4D8C199D0983
:1071C0000817190708F049C081E0F7018483782A7D
:1071D000BFEF8B1A9B0AE7E0EE0EF11CF0E28F1670
:1071E000910409F083CF611409F418C1711409F4F2
:1071F00015C10E945A4D9093371380933613809196
:107200003513883030F591E0980F9093351399E05D
:10721000FE013A96DE01119601900D929A95E1F7E2
:107220002DE0829FC001112483539D4E29E0FE0171
:107230003196DC0101900D922A95E1F72FEF3FEF97
:10724000DC011A963C932E9319971C96BC92AE9231
:107250001B976C96E2E10C942F5F2091CC128091E9
:10726000CB12922F40E050E0281709F448C0C22EFC
:10727000D12CF601EE0FFF1FEF53FD4E008111815F
:1072800037E0309FF001319FF00D1124EF51FE4E99
:10729000408151815C8F4B8FB0E030E0A0E0EB8DFE
:1072A000FC8DEA0FF11DEA0FF11D4081518141155E
:1072B0005105E1F0F7010190F081E02DFA8FE98F9F
:1072C00030E007C0E1E04617570709F0E0E0BE2BC9
:1072D0003F5FE98DFA8DE30FF11DE30FF11D608132
:1072E00071816115710571F7AF5FD9CFB11599F152
:1072F0003A17C8F4E1E0D7011496EC93A7019093F4
:10730000CC124E155F0569F090E0FC01EE0FFF1FF7
:10731000EF53FD4E9182808201968370992780936E
:10732000CB12852D54CFF7E0F09FA001F19F500DB7
:1073300011244F515E4EE1E0DA011496EC934E15A4
:107340005F05E1F2291302C09F5F937096012F5FE2
:107350003F4F237089CF40E050E0F8CF292F30E035
:10736000411022C0B10102C0660F771F8A95E2F773
:10737000CB0101972817390789F0512CF10102C080
:10738000EE0FFF1FCA94E2F76F01C094D701169663
:107390008C9116978C2116968C93C3CF411571F35F
:1073A000C4010E94830CE9CFA9010C2C02C05595A1
:1073B00047950A94E2F7C901019782239323892B09
:1073C00039F540FF25C0D70112968D919C91892BEC
:1073D000D1F087E0FE013196DF011D928A95E9F731
:1073E0000E945A4D9C018B839C8384E08D83F7011E
:1073F00092818381792F9887898709811A8144E056
:107400005E816F8153DCD70115961C92542CB6CF48
:10741000B42FB1705B2EB2CF80E0D9CE9091CC1258
:107420008091CB12981731F00DDDB1E07B1609F495
:1074300010CF2FCEB6DC10923713109236130E9465
:10744000720CF3CFA6E0B0E0E8E2FAE30C94215F1F
:107450000E945A4D8C018091E60B9091E70B8017AA
:10746000910771F019821A820E945A4DBC0149811C
:107470005A8180E090E093DD1093E70B0093E60BD8
:107480002696E4E00C943D5FCDB7DEB7EC970FB6DF
:10749000F894DEBF0FBECDBF85B7806885BF85B7C6
:1074A000806885BF1092700A1092720A1092710A59
:1074B00080EC8093350B83E79AE09093370B8093B1
:1074C000360B1092340B1092330B1092500A10921C
:1074D0004F0A1092520A1092510A1092540A1092B6
:1074E000530A1092560A1092550A1092580A109296
:1074F000570A10925A0A1092590A10925C0A109276
:107500005B0A10925E0A10925D0A1092600A109255
:107510005F0A1092620A1092610A1092640A109235
:10752000630A1092660A1092650A10926A0A109213
:10753000690A8FE591E190934C0A80934B0A8FE1A1
:107540009EE090936C0A80936B0A88E390E290939C
:10755000680A8093670A81EE99E090934E0A8093BF
:107560004D0A84B7877F84BF0FB6F894A8958091A1
:107570006000886180936000109260000FBE80E818
:1075800090E00FB6F89480936100909361000FBE75
:1075900081E0809379028AE598E090939505809345
:1075A00094050E94A50B0E949A0F0E94E10F0E9471
:1075B00060100E94B10E0E944F4E0E94F44D8091C7
:1075C000E20084608093E20078948091E10B811561
:1075D00099F08091E9001091EC008F7017951127B8
:1075E0001795182B1092E9008091E80083FD0E9406
:1075F0005D4F1F701093E90082E084BD93E095BD5C
:107600009AEF97BD80936E000E94170F811102C000
:107610000E94FF1B80E30E941D1487EC0E941D1432
:1076200080EF0E941D1481EF0E941D140AE414E0F3
:1076300046E5E42E44E0F42ED8018D918D018F3F74
:1076400011F00E941D14E016F106B1F788E0E7ED95
:10765000FBE0DF01282F1D922A95E9F7E7EEF8E01D
:10766000DF011D928A95E9F7569A5E9A80E090E0D4
:107670000E942160833E9E4F21F40E94170F8111CA
:1076800002C00E94251C82E090E00E941960809355
:10769000EF0884E090E00E94216090936313809350
:1076A00062130E944F59EFEFF6E721E0E150F040FE
:1076B0002040E1F700C000000E944F598091D70B95
:1076C00080FF08C06FEF7FEF80E090E00E944F6086
:1076D0000E949F4D83E090E00E9419600E947F0508
:1076E0000E945F140E945F1210921C0A40E150E059
:1076F0006FEF70E085E39AE00E9402601092050946
:1077000040E150E06FEF70E08EE199E00E9402608E
:1077100081E08093450A48E050E067E170E08FEC3B
:107720009BE00E9409601092450A8091CF0B843043
:1077300010F40E94B81188E292E09093090C8093B3
:10774000080CAE014F5F5F4F5CA74BA75BA55DAB1D
:107750008CA58EAB0E944F59A0EFB8E0B8ABAFA795
:10776000E7EDFBE0FAABE9ABDF01E0EFF8E02191F8
:1077700031918D919D9148EF58E04E175F0709F4C4
:1077800098C02817390799F387ED9BE09CAB8BAB2A
:10779000C12CD12C00E0EBA9FCA921903190FCABCD
:1077A000EBABAFA5B8A98D919D91B8ABAFA78215F2
:1077B000930509F435C1FC01E225F325F8AFEFABE1
:1077C000DEA6CDA6712C44244394512C8FA998ADEC
:1077D00084219521892B09F413C15101A420B520DE
:1077E00079820A830E945A4D9C838B83F1E0FD834A
:1077F00091E0A114B10409F490E09E8349815A817B
:107800006B817C818D81CBDB10E0A114B104B1F0E0
:10781000033009F086C025E0721283C08AE28983B2
:1078200011E0EDA5FEA5EA5AFB4F80818F3F31F0B4
:10783000FE013196E10FF11D80831F5F6091050904
:10784000E12EF12C412F460F5527551F4930510588
:107850005CF188E0882E912C8E189F08B7016A5F32
:10786000764FA40186E099E00E94E85FB701625F6D
:10787000764FA4018EE099E00E94E85FA401440FD6
:10788000551FB701660F771F625E764F8EE199E054
:107890000E94E85FB7016A5E764FA40186E199E035
:1078A0000E94E85F68E0611BAE014F5F5F4F70E0D0
:1078B0005BC02817390781F5C5DD80910409811166
:1078C0000EC000910209109103090115110509F07C
:1078D000ECC00E945A4D9093030980930209809155
:1078E000CC0D811509F409C10091C80D1091C90D85
:1078F0000115110509F0F5C00E945A4D9093C90D6C
:107900008093C80D8091CA0D282F30E0811509F4AD
:1079100010C2C901019711C2A7EDBBE0BCABABAB74
:1079200037CF10E07ECFDA01FD90AD012F2D30E092
:1079300090E0FC01EB5FF64FD901AA0FBB1FAA57DD
:10794000BB4FAC91A183220F331FD901AA5ABB4F61
:10795000D1962C912187F18AFC01EE0FFF1FEB5F7E
:10796000F64F128E118E7F5F872F860F1713DBCF96
:1079700080930509AB2809F443C08091CF0B8C7F1D
:107980008C3709F03DC0EDA5FEA5EA5AFB4F80817A
:107990008F3FB1F1A12CB12C612C90E09C01220F02
:1079A000331FF901EA57FB4FFAAFE9AF29573B4FB5
:1079B0003CAF2BAF4DA55EA54451564F4A01750112
:1079C00010E0F701EA5AFB4F80818F3F59F0061112
:1079D00031C071122FC0D4012C9130E2230F08F472
:1079E0002FEF2C931F5FBFEFEB1AFB0A1C3049F7F8
:1079F0006394ECE0AE0EB11CF0E3AF16B104F9F6FF
:107A00007394440C551C2DA53EA52F5F3F4F3EA7F8
:107A10002DA73CE07312DACEEFA5F8A9329222929C
:107A20000F5F4CE0C40ED11C043009F0B4CE0E94AC
:107A30006F4D43CF90E0E9ADFAAD4081FC01EE0F10
:107A4000FF1FEA57FB4F2081421B550BABADBCAD6E
:107A50002C91880F991FFC01EA5AFB4F81A9281B22
:107A6000330B449FB001459F700D700D1124229F70
:107A7000C001239F900D900D1124860F971F0E9427
:107A80004117382F893208F0ADCF28E2231B08F4C4
:107A900020E0F701E451F64F213108F020E1308178
:107AA000320F08F43FEF30839DCF0E945A4D801B68
:107AB000910B8D32914008F412CF8091B60D80FF6A
:107AC00006C065E070E084E392E00E9460570E9487
:107AD0005A4D9093F9088093F80881E08093040947
:107AE000FECE0E945A4D801B910B20913C03309199
:107AF0003D032817390708F4FFCE0091BA0F109103
:107B0000BB0F0115110591F1C090FE08D090FF0840
:107B1000E0900009F09001090E946F4D6C197D09F9
:107B20008E099F09C090FA08D090FB08E090FC08ED
:107B3000F090FD086C157D058E059F05B8F0C80115
:107B40000E94461A1092BB0F1092BA0F1092FE08B4
:107B50001092FF0810920009109201091092FA0881
:107B60001092FB081092FC081092FD08E090C211E0
:107B7000F090C311E114F10439F1C090C411D09018
:107B8000C5110E945A4D8C010C191D09C7010E9494
:107B9000D25880179107C0F42091C2113091C311BF
:107BA000C9019927207E3327232B09F0DFC024E069
:107BB000880F991F2A95E1F78E53904FDC01159697
:107BC0002C9122FF0E949A1C8091A003811511F133
:107BD000009136131091371301151105D9F00E9449
:107BE0005A4D801B910B2091C9123091CA1228174F
:107BF000390780F49091CC128091CB12981709F438
:107C0000B8C020D91092CA121092C912109237131C
:107C1000109236138091551380FF1CC080913F0352
:107C200082FF18C00E945A4DBC018091C6119091EC
:107C3000C7119B01281B390B80915C0290915D025A
:107C40002817390738F041E08091C8119091C91187
:107C50000E9443588091D10D811569F00E945A4DC0
:107C60002091D20D3091D30D821B930B8F3F9F47F4
:107C700010F40E949D19C0902E09D0902F09E09019
:107C80003009F09031090E946F4D2B013C015301E6
:107C900042018C189D08AE08BF080E946F4D60938A
:107CA0002E0970932F098093300990933109A09188
:107CB0000509E5E0F9E04A2F50E02FEFC20ED21E91
:107CC000E11CF11CC418D508E608F708A51359C033
:107CD0004093050920914A0A412C21110AC02091A4
:107CE000CF0B322F3370432E311519F0422E4694AC
:107CF000469420916902223009F4A3C608F051C0CD
:107D00002111D2C0109264026093460A7093470A10
:107D10008093480A9093490A89E2E5E0F9E0ACE1F2
:107D2000BAE001900D928A95E1F781E080936902B3
:107D30003BC08091CB0D8150990B2854324FD90113
:107D40001C918854924FFC0180810E941215812F52
:107D50000E94FC1F8091CA0D90E001966091CB0DAE
:107D600070E00E944A5F8093CA0DC7CE80E090E029
:107D700025CF17D810923713109236130E94720C29
:107D800049CF218D328DC216D306E104F10420F4CF
:107D900041505F5F32969ACF280D391D328F218F67
:107DA000F8CF233009F457C6E0916B0AF0916C0AC2
:107DB000309719F08BE49AE009959FB7F8940091F9
:107DC000340B8091330B081708F461C6081B9FBF62
:107DD000E12CF12C10E0CC24C394D12C9924939461
:107DE000E016F10608F457C60E94CD188091E10B09
:107DF0008430E1F480916B028F708093E900909160
:107E0000E80090FF13C09091E10B943079F48093D7
:107E1000E9008091F2009091F300892B39F0809174
:107E2000E8008E778093E8000E94C34D8091E10BBB
:107E3000843009F08FCC83E08093E9008091E800E2
:107E400082FF88CC8091E80090E085FF09C040E087
:107E500050E060E270E08DA99EA90E94E95291E095
:107E60008091E8008B778093E800911509F472CC3B
:107E70000091E40B1091E50BE9810115110509F45E
:107E8000C3C6EE3F09F0E3C68A81833020F08550F7
:107E9000833008F0DCC6EA81EE3008F0D8C6F0E0A6
:107EA000EC5AFE490C945D5F80916802481223C031
:107EB0009091CF0B93702091670230E081E0921790
:107EC000130609F480E0809366028091D40B9091B0
:107ED0006502981739F08093650240E060E080E029
:107EE0000E94DE0A4EE2441688F4E42DF0E0EE59DA
:107EF000FE490C945D5F81E0E6CF809166028115BA
:107F000029F040E060E080E00E94DE0A80E0E7C007
:107F1000809164020E942518082FF92E6091D00BE1
:107F20007091D10B8091D20B0E947D15E62ED72E39
:107F3000C82E10E0F01609F020F481E051E3F516A8
:107F400038C0F801E851FB4F808190916502892388
:107F5000811531F02C2D4D2D6E2DC8010E94221857
:107F60000F5F1F4FE7CF809164020E942518082FF2
:107F7000F92E1091D00BA090D10BB090D20B612FA5
:107F80007A2D8B2D0E947D15E62ED72EC82E80913E
:107F9000D30B612F680F7A2D8B2D0E947D15B62E85
:107FA000A72E982E10E0F01609F030F481E091E34E
:107FB000F91608F494C0AACFF801E851FB4F90815C
:107FC000809165028923811559F0292D4A2D6B2D49
:107FD00090FD03C02C2D4D2D6E2DC8010E9422183E
:107FE0000F5F1F4FE0CF809164020E942518082F79
:107FF000F92ED090D10BC090D20B6091D30B80E4BE
:108000000E940416E82E10E0F01609F020F481E03A
:10801000A1E3FA16CECFF801E851FB4F8081909191
:10802000650289238115B1F0F801EE0FFF1FEA5AAE
:10803000FB4F81A982958F706091D00B8E9D600D52
:1080400011247D2D8C2D0E947D15472F282FC801CE
:108050000E9422180F5F1F4FD7CF809164020E94A9
:108060002518082FF92ED090D10BC090D20B60911B
:10807000D30B80E40E940416E82E10E0F01609F0FD
:1080800020F481E0B1E3FB1694CFF801E851FB4FF7
:1080900080819091650289238115D1F0F801EE0F5E
:1080A000FF1FEA5AFB4F80A98E9DC0011124B5E045
:1080B00095958795BA95E1F76091D00B680F7D2D66
:1080C0008C2D0E947D15472F282FC8010E94221851
:1080D0000F5F1F4FD3CF8DE098E10E946E559091B6
:1080E00064029F5F9093640281115ECE82E0809370
:1080F000690280916602811157CE411055CE83E00E
:1081000015CE8AEE96E1E9CF83EB96E1E6CF86E9DC
:1081100096E10E94F753E3CF8AE796E1FACF8FE525
:1081200096E10E944F54DBCF85E496E1FACF8FEDC4
:1081300099E0D3CF86ED99E0D0CF8DEC99E0CDCF0B
:1081400084EB99E0CACF83EA99E0EBCF81E797E12E
:10815000E0CF88EC9AE0DDCF85EB9AE0E2CF85E7CF
:1081600099E00E94B654BBCF86E499E0FACF8DE047
:1081700099E0F7CF1091640211111AC06091D30BEE
:1081800020E1620F08F46FEF8091460A9091470A50
:108190000E9422176AE070E00E94FF5E892B41F482
:1081A00081E30E94AE1790E090935F0280935E029D
:1081B000812F0E942518282F192F082F80916602E1
:1081C000811117C080915E0290915F028217910524
:1081D00090F08117910578F40E940C5582E390E0AD
:1081E00090935F0280935E0206C0802F0E940C5520
:1081F0000F5F0117D0F381E01133DBCE10916402E1
:1082000011111AC06091D30B20E1620F08F46FEFD7
:108210008091460A9091470A0E94221765E070E01B
:108220000E94FF5E892B41F481E30E94AE1790E02B
:108230009093610280936002812F0E942518282F5D
:10824000192F082F80916602811117C0809160025A
:10825000909161028217910570F28117910558F68D
:108260000E944A5582E390E09093610280936002FD
:10827000C2CF802F0E944A550F5F0117D0F3BBCFAA
:1082800086EF97E12ACF86ED97E127CF8BE296E143
:1082900024CFF0906402F1101FC0009132091091B8
:1082A00033090E945A4D4091D30B20E431E0241B46
:1082B0003109801B910B2817390770F481E30E9464
:1082C000AE1790E090936302809362020E945A4D31
:1082D00090933309809332098F2D0E942518F92E2F
:1082E00000916202109163020817110540F109170D
:1082F000110528F5F801E851FB4F80819091650246
:1083000089238115E1F00E94991781FD1CC00E940C
:108310009917E82E80E80E94AE177FE7780F8091CA
:10832000D20B6E2D0E947D15472F282FC8010E9469
:10833000221882E390E0909363028093620281E0CE
:10834000E1E3FE1636CE80E070E0E12CEACF8091CA
:10835000C7099091C809A091C909B091CA09409173
:10836000460A5091470A6091480A7091490A481795
:1083700059076A077B0708F4C9CD8091660281110D
:1083800054C0809164020E942518D92E082F10E055
:108390007801EE0CFF1CE00EF11E97012C5C364FAD
:1083A00079010D1508F46FC0E1E3DE16D0F18D2DD3
:1083B00090E07C01F1E0EF1AF108AC01440F551F89
:1083C000480F591F4350510967E379E084E399E06E
:1083D0000E94F15F0E9499178701000F111F81FF12
:1083E0006CC00E0D1F1DF801EC5CF64F108211825F
:1083F00012820E942F170091460A1091470A20917D
:10840000480A3091490ADC01CB01800F911FA21F5D
:10841000B31F8093C7099093C809A093C909B0936B
:10842000CA0981E021E3D216C4CD40E060E080E0DB
:108430000E94DE0A04E319E0E7ECEE2EE9E0FE2EEE
:108440000E94991781FF0DC0D8011C9211961C92B1
:10845000119712961C920D5F1F4FE016F10681F7DF
:1084600090CF0E949917D82E80E80E94AE177FE720
:10847000780F6D2D8091D20B0E947D15F8016083DD
:1084800071838283E8CFF801E851FB4F808190919E
:1084900065028923811559F0D70112962C91129704
:1084A00011964C9111976C91C8010E942218B3E06B
:1084B000EB0EF11C0F5F1F4F74CF0E949917C82E4F
:1084C00080E80E94AE177FE7780F6C2D8091D20B69
:1084D0000E947D150E0D1F1DF801EC5CF64F6083A8
:1084E0007183828386CF80916602811529F040E0F6
:1084F00060E080E00E94DE0A809164020E942518FC
:108500009BAB8091460A9091470AA091480AB0918E
:10851000490A4091E3095091E4096091E50970919D
:10852000E609481759076A077B0708F0AAC0609157
:10853000D00B7091D10B8091D20B0E947D15B62E7D
:10854000A72E982E0BEC19E046E5E42E44E0F42E1D
:1085500017012CE0E20EF11C3EA62DA6F8AAEFA60C
:108560006801712CD6018D916D01892C5A2C6B2CD0
:10857000811103C0812C512C612CEDA5FEA58191A8
:10858000FEA7EDA790E0FC01E851FB4F2081309160
:1085900065022323211529F0282D452D662D0E94E3
:1085A0002218AFA5B8A98E91B8ABAFA790E0FC0197
:1085B000E851FB4F2081309165022323211529F0DA
:1085C000282D452D662D0E942218F6018081829368
:1085D0007394F5E07F12C6CFD80115968C91792C53
:1085E0006501811103C0712CC12CD12CF101858151
:1085F00090E0FC01E851FB4F20813091650223237C
:10860000211529F0272D4C2D6D2D0E942218D10106
:1086100016968C9190E0FC01E851FB4F208130913F
:1086200065022323211529F0272D4C2D6D2D0E9445
:1086300022180E949917837091E0811190E0F8014F
:1086400095830A5F1F4FF6E8EF16F4E0FF0609F086
:108650007FCF0E942F170091460A1091470A209160
:10866000480A3091490ADC01CB01800F911FA21FFB
:10867000B31F8093E3099093E409A093E509B093B5
:10868000E60981E03BA9313394CC809164020E94D9
:108690002518682ED92E80916602811561F040E080
:1086A00060E080E00E94DE0AECEEF9E080E3DF01AA
:1086B0001D928A95E9F780916402811117C000919B
:1086C000E8091091E9090E945A4D801B910B21E0A5
:1086D0008931910508F420E02093E709499730F0AB
:1086E0000E945A4D9093E9098093E809812C912CBE
:1086F000712C3AEA532E54012CE0C22EF501EA5AAD
:10870000FB4FE080E61408F43BC0ED1408F038C0DD
:10871000F12CF701E851FB4F80819091650289238C
:10872000811569F1F501E451F64F1F011081012F08
:1087300025E5021B08F400E03091D10B3DA7252D63
:10874000210F08F42FEF822F880F820F6091D20B38
:108750008E5F0E940416652D601B7DA50E947D150D
:10876000472F282FC7010E9422188091E709811501
:1087700031F041E0141B08F410E0D1011C93739414
:10878000CA94BFEFAB1ABB0AC110B8CFE4E28E1691
:10879000910421F481E031E3D3160BCCFCE08F0E81
:1087A000911C2AE0721608F4A6CFF4CF5090D20B99
:1087B000A52CB12C8501000F111F0A0D1B1D16954C
:1087C0000795169507950DA78FEF90E0B5010E94CC
:1087D0004A5F362E80916602811571F040E060E0BC
:1087E00080E00E94DE0AECEEF9E080E3DF011D92FA
:1087F0008A95E9F71092EB098091EA098F5F8093DF
:10880000EA09BCEE8B2EB9E09B2EC12CD12CF501D0
:10881000E01BF10BF8ABEFA736017401212C80911E
:10882000EB09822981112FC00E94C45F85359540D4
:1088300054F5D4015C9280E0F301EA5AFB4F908139
:108840009F3FB9F1FE013196E80FF11D9083D701EA
:108850002C91E981F0E0BDA5B21708F04FC030E0DF
:10886000201B310B209FC001219F900D309F900D48
:1088700011246FA578A90E94FF5E262F452DCF01F8
:108880000E94221818C0F7018081811541F08515DA
:1088900030F49091EA09391202C081508083F3E0EC
:1088A0002F12C9CF25E0C212C6CF3AE2398381E048
:1088B000C3CF8111CCCF2394ECE0EE0EF11CFCE091
:1088C0006F0E711C24E02212AACF3FEFC31AD30A05
:1088D0004FEF841A940A5CE0C516D10409F09CCFCE
:1088E0008091EA09381202C01092EA098091EB09DE
:1088F0008F5F8D3178F48093EB0908CB2A9DC001FE
:108900002B9D900D1124B8010E94FF5E462F20E0A0
:1089100060E0B5CF1092EB0984E09AE063E028EFC5
:1089200039E07FEF750D8C01ECEEF9E0633021F456
:1089300044A1541201C074A3D8014D918D01451575
:1089400040F0AD0141505109DA017C93D8011B96EA
:108950005C9231962E173F0749F761500C976111D1
:10896000E2CFD4CA8EE196E10E94B255B8CB8CE03A
:1089700096E1FACF80911C0A21E0382F321B08F4CF
:1089800030E0832F64EF78E00E941F56A8CB64EF9D
:1089900078E080E0F9CF80911C0A21E0482F421B4B
:1089A00008F440E0842F6CEB78E0EECF6CEB78E0DD
:1089B000F0CF80911C0A21E0582F521B08F450E0A0
:1089C000852F6AE878E0E0CF6AE878E0E2CF80912E
:1089D0001C0A21E0382F321B08F430E0832F62E7B5
:1089E00078E0D2CF62E778E0D4CF80911C0A21E012
:1089F000482F421B08F440E0842F6CE578E0C4CF98
:108A00006CE578E0C6CF809164020E942518F92EAB
:108A1000082F10E00F1508F090CAF801EE0FFF1FA5
:108A2000E00FF11FE45CF44F6081718182810E944C
:108A30007D15472F282FC8010E9422180F5F1F4F56
:108A4000E9CF409268028091CF0B837080936702D8
:108A50000E941F1254CB8091450A81110E94AD11D2
:108A6000C090460AD090470AE090480AF090490A20
:108A70000E946F4D6C197D098E099F096031710547
:108A80008105910508F490C9109269028DC9209161
:108A9000350B020F9BC98091330B90E06091350B31
:108AA00070E00E944A5F2091360B3091370B280FFF
:108AB000391FD901BC90A090700AB8EFBB16E8F03E
:108AC0009092700A20E040E06B2D81E090E00E94DF
:108AD0001F53A092700A2FB7F8948091330B90E047
:108AE00001966091350B70E00E944A5F8093330BD2
:108AF0002FBF4FEFE41AF40A73C9B7FE54C0E4E085
:108B0000AE1631F0B0926D0AD092720AC092710A1C
:108B10008B2D0E94570A823081F0833071F08130B2
:108B200079F48093700A20E040E06B2D81E090E0C2
:108B30000E941F531092700ACECF8093700ACBCF41
:108B4000F0EFBF1651F027EFB21699F01092700AAD
:108B50001092720A1092710ABECF84E08093700A5C
:108B6000B0926D0A81E090E09093720A8093710A4E
:108B7000B2CF2091710A3091720AC90163E070E0AE
:108B80000E94FF5EFC01E55BF54FB2A2C9010196B0
:108B90009093720A8093710A20916F0A40916E0A35
:108BA00060916D0AC5CFA11409F495CF2091710A87
:108BB0003091720AC90163E070E00E94FF5EAC016F
:108BC000FC01E55BF54FB2A2C90101969093720AD0
:108BD0008093710A4130510591F04230510509F0FE
:108BE0007ACF20916F0A40916E0A60916D0A0E94BF
:108BF0001F538091700A843009F0B4CF6CCF32E0FB
:108C000020E0A31268CFEFCFE43150F4E11559F022
:108C1000E150E33140F4F0E0E057FE490C945D5F31
:108C2000EE3F09F438C98FEF1CC51A8289E08B83A7
:108C30000EC08A81823089F08330C1F0813099F78B
:108C40004ED70E94765F6B837C838D839E838DA934
:108C50009EA90E9411530C94AA3B88E290E00E94C6
:108C600019601B821C821D828E83F1CF8091DF0BE5
:108C70009091E00B892B59F3FE0131968FED9BE02B
:108C8000A9A9BAA92C9111963C9111971296BAAB49
:108C9000A9AB3283238332968A179B0789F7D7CFF4
:108CA0008A81823009F0BFCF6B817C818D819E816A
:108CB0000E94765F88E290E00E943560C8CF4C81C8
:108CC0006B818A810E94D70E9827892798279E83D7
:108CD0008D83BDCF2D813E813227232732274C81C2
:108CE0006B818A810E94D70DB2CF0E94601BAFCFEB
:108CF0008A818134B9F1823409F0A9CF8D8190E065
:108D00009C01220F331F280F391F2E3131050CF023
:108D10009ECF4B815C81DE011196FA01EE0FFF1FA1
:108D2000E40FF51FE45CF44F20E030E0281739072A
:108D300008F08DCF1396B901640F751F613371056B
:108D400008F085CF12966C911297608313966C9100
:108D50001397618314966C91149762832F5F3F4F32
:108D60003396E4CF0B811C810115110581F40E941B
:108D7000F80A8D818093D30B80E00E94D80A8E81FF
:108D800020E048856F8190E00E94330B60CF0E9405
:108D9000EA0A24E036E048EB56E0F9013296859184
:108DA0009591F901659175916017710731F02C5F0C
:108DB0003F4F4217530789F780E060E00E94040BA1
:108DC000D8CF8A81823409F46CC0A8F5803409F4C4
:108DD00062C0813409F03BCF8091CF0B982F937004
:108DE0009115C1F08695869590E024E036E068EB19
:108DF00076E0F9013296A591B591F9014591559129
:108E0000E42F452F8A179B0739F02C5F3F4F6217DD
:108E1000730779F7E0E040E0EB834C838091D30B5C
:108E20008D838091D00B8E838091D10B8F83809125
:108E3000D20B88870CCF833409F456C0843409F0F0
:108E400006CF8B81282F30E0813308F000CFF90165
:108E5000EE0FFF1FEA57FB4F80818B83F901EE0F66
:108E6000FF1FEA5AFB4F81A98C83F901E851FB4FA0
:108E700080818D838FEF8F838E8366E574E040E081
:108E800050E0FB0180E090E0A191A217130681F56C
:108E90004E838F83DCCE81E08B831C828FEF8D83AA
:108EA000D6CE0B811C814EE150E06FEF70E0CE0119
:108EB00003960E94026084E096E048EB56E0DE01F3
:108EC00013966EE1FC01259135910217130728F4E2
:108ED000623040F02D933D93625004964817590735
:108EE00089F7B5CE60E0F9CF81E38B831C82AFCEEA
:108EF00001968C30910541F64F5F5F4F645F7F4F65
:108F00004430510509F0BDCFA2CE0E94AD119FCED5
:108F100080E18A839CCE88E08A838FE288CE0C81B0
:108F20000D3108F094CE8A809B809824892498245F
:108F3000A12CB12CFE0131967F010E0F1F2F111DA8
:108F40000E151F0509F483CE80E0FFE28F16F8E0CE
:108F50009F06A104B10428F4C4018F52984F0E94C7
:108F60001960D70114968C93BFEFEB1AFB0AEFEF51
:108F70008E1A9E0AAE0ABE0AE3CF8091DF0B909153
:108F8000E00B892B09F463CE8C818D3108F05FCE24
:108F9000882E912CA12CB12CCA80DB80DC24CD241E
:108FA000DC24E12CF12C8E010F5F1F4F412C512C42
:108FB0003201481459046A047B0408F048CEFFE2E9
:108FC000CF16F8E0DF06E104F10440F4D80114966E
:108FD0006C91C6018F52984F0E943560BFEF4B1ABB
:108FE0005B0A6B0A7B0AEFEFCE1ADE0AEE0AFE0A74
:108FF0000F5F1F4FDECF0E94CA1129CE88E089CFB4
:109000008C818D3108F023CE882E912CA12CB12C8F
:10901000CA80DB80DC24CD24DC24E12CF12C412C23
:10902000512C32018E010B5F1F4F481459046A0402
:109030007B0408F00CCE80E0C114F3E0DF06E1040D
:10904000F10420F4C60189960E941960D8018D931D
:109050008D01BFEF4B1A5B0A6B0A7B0AEFEFCE1A4A
:10906000DE0AEE0AFE0AE1CF2C81022F10E02D313C
:1090700008F0EDCD8A819B819827892798272C01BC
:10908000612C712C8115F3E09F0708F0E0CD822E52
:10909000912CA12CB12C40E053E060E070E0441929
:1090A000550966097709421751056105710508F4EC
:1090B000CECD2091DF0B3091E00B232B09F040C087
:1090C0001C0129E2220E311C80FBEE24FF24E0F873
:1090D00080FF0CC088960E9419609D81892798277F
:1090E000892781159C4711F48FEF8D83D501C40129
:1090F000840D951DA61DB71D80FF1AC0680141E0B3
:10910000C41AD108CE0105968C0D9D1D9EA78DA772
:10911000C101800F911F0E941960ADA5BEA59C9151
:1091200081159C4721F48FEFEDA5FEA58083860174
:10913000FE013196EE0DFF1D2FEFE016F10638F01F
:109140008E010F5F1F4FC12CD12C760125C0948159
:10915000858181159C4711F42483258342E0E40E28
:10916000F11C3296EACF411453E0550661047104B4
:1091700038F4D80114966C91C20189960E9435602A
:10918000BFEFCB1ADB0AEB0AFB0AEFEF4E1A5E0ABF
:109190006E0A7E0A0F5F1F4FC814D904EA04FB044D
:1091A00010F355CD8091DF0B9091E00B892B09F4E2
:1091B0004ECDCE0101960E941153FFEF21EE34E017
:1091C000F15020403040E1F700C00000B8D43FCD5E
:1091D00088E0EFEDF3E0DE01919601900D928A9523
:1091E000E1F7FE0132968FE1DF011D928A95E9F7E2
:1091F00086E0898388E07F96DE01159601900D92C6
:109200008A95E1F781E08D8722CD8CE5898381E025
:109210008A831B826BCE8B819C81092E000CAA0B4A
:10922000BB0B35E0880F991FAA1FBB1F3A95D1F7DA
:10923000AC01BD01405E5F4F6F4F7F4F481759072C
:109240006A077B0708F403CD8C35E1E09E07A10592
:10925000B10508F0FCCC4D35F1E05F076105710503
:1092600020F04CE551E060E070E0481B590BBC0178
:1092700068557B4FCE0101960E94D25FE8CC4AE14F
:1092800050E06FEF70E0CE0107960E94026080917F
:10929000DF0B89830A831B821C8283E08D8385E038
:1092A000E3CC81E090E09093E50B8093E40B82E3C4
:1092B00090E090933B0B80933A0BFCD39093390B47
:1092C0008093380BC4CC0115110571F1D090D70BE8
:1092D000C090DD0BE090380BF090390BEBD38E197A
:1092E0009F098536910538F1C5FE25C0D0FE23C003
:1092F000E1D39093390B8093380B80913A0B909186
:109300003B0B019790933B0B80933A0B892B61F4B5
:109310001092E50B1092E40B81E090E09093E00B4B
:109320008093DF0B00E010E08091DF0B89830A83DC
:1093300080913A0B7CCC82E390E090933B0B80933E
:109340003A0BF2CF1092E00B1092DF0B80CC0B8126
:109350001C8140E250E06FEF70E0CE0101960E9468
:1093600002602CED33E042E050E080E090E0F90153
:10937000659175910617170740F4DE0111968A0F63
:109380009B1FFC0171836083CA01F4E02C393F0705
:1093900009F45DCCAC014E5F5F4F245F3F4F41321B
:1093A000510528F354CC4B815C818CED93E028EA85
:1093B00034E0FC01659175914617570709F442C1E5
:1093C0000C9628173907A9F72ECC8B819C810CEDC0
:1093D00013E0F801259135918217930709F443C1F1
:1093E000045F1F4FF4E0083A1F0799F7EE24EA9450
:1093F000FE2C54C10E942D1B2ACCEB81E93008F0D1
:1094000026CCF0E0ED55FE490C945D5FFE013596EB
:109410008BE1DF011D928A95E9F780E289838A83D7
:109420008B838C8383E088A312CC8C819AE0F92E05
:109430008E010F5D1F4FF8012F2D11922A95E9F72C
:10944000B8010E9454188983F801DE011296019038
:109450000D92FA94E1F7FBCB1C818AE0FE01359670
:10946000DE01919601900D928A95E1F789A19AA16A
:109470000E94980B9AA389A38BA19CA10E94980B90
:109480009CA38BA38DA19EA10E94980B9EA38DA34C
:109490008FA198A50E94980B98A78FA38FEF1032E9
:1094A00068F43AE0139FB00111246F5A7C4F4AE0F0
:1094B00050E0CE0181960E94536080E089830E9433
:1094C000A50BC5CB2C816AE0CE018196DC01E62F8D
:1094D0001D92EA95E9F7203208F04AC0629FB00178
:1094E00011246F567B4F4AE050E00E94096080E0F3
:1094F00089838AE0FE01B196DE01129601900D92F9
:109500008A95E1F7A4CB1C818AE0FE013596DE0145
:10951000919601900D928A95E1F789A59AA50E94EE
:10952000980B9AA789A78FEF103268F4FAE01F9F73
:10953000B00111246F567B4F4AE050E0CE01819676
:109540000E94536080E089830E949A0F80CB2C8117
:109550006AE0CE018196DC01E62F1D92EA95E9F7DB
:10956000203230F4629FB00111246F527A4FBBCF8A
:109570008FEFBECF1C818AE0FE013596DE01919609
:1095800001900D928A95E1F78BA19CA10E94980B06
:109590009CA38BA38FEF103268F4FAE01F9FB001F9
:1095A00011246F527A4F4AE050E0CE0181960E941A
:1095B000536080E089830E94E10F49CB2C8166E0F3
:1095C000CE018196DC01E62F1D92EA95E9F7203263
:1095D00068F4629FB00111246F5E784F46E050E05E
:1095E0000E94096080E0898386E084CF8FEFFBCF03
:1095F0001C8186E0FE013596DE01919601900D9268
:109600008A95E1F789A19AA10E94980B9AA389A350
:109610008BA19CA10E94980B9CA38BA38FEF10326F
:1096200068F4F6E01F9FB00111246F5E784F46E0AA
:1096300050E0CE0181960E94536080E089830E94B1
:10964000601005CBFC013696259135912115310529
:1096500009F4E9CA4FE150E0BE016E5F7F4FF901A6
:1096600009958983F4CAF801389625913591211519
:10967000310509F4BBCE4CE150E0BE016B5F7F4F7A
:10968000C801F90109957C01892B41F4F8013A964A
:1096900085919591009711F0FC010995E982D7CA4F
:1096A000A6E0B0E0E6E5FBE40C94235F9093E30BC7
:1096B0008093E20B811520E2920730F40E94461A53
:1096C0002696E2E00C943F5F80EF89838A83F2D193
:1096D0008160BC0149815A8181E091E00E94CF37CD
:1096E000EFCF0F931F93CF93DF938C01862F6CEAFC
:1096F0007DE00E945418892BA9F4C091AC0DD09143
:10970000AD0D209779F0F8018281833051F4CE01BC
:109710000E94AF22CE010E94AF22CE010E94AF2252
:1097200001C0D8F7DF91CF911F910F9108950F934A
:109730001F93CF93DF938C01EB016CEA7DE08C2FBC
:109740000E945418892B09F059C0FE01FF27D80147
:1097500012968C911297EC5DF84F8130A9F4159612
:109760008C9182FD50C080FF4EC082E0808380914A
:10977000AE0D9091AF0D0097B9F48091AC0D909122
:10978000AD0D0097D9F110C08230B1F515968C91CE
:1097900082FD27C080FD0AC083E080838091B00DE8
:1097A0009091B10D0097F9F07BDF28C084E08083B1
:1097B0008091B20D9091B30D0097B1F78091AC0DEF
:1097C0009091AD0D009711F10E94AF228091AE0DE6
:1097D0009091AF0D009741F78091AC0D9091AD0D38
:1097E000E3CF85E080838091AC0D9091AD0D009723
:1097F00029F00E94AF22F0CF86E08083DF91CF91E5
:109800001F910F91089581E08083B7CF8091AE0DB5
:109810009091AF0DB6CF0F931F93CF93DF938C0131
:10982000EB016CEA7DE08C2F0E945418892BA1F487
:1098300080915813909159130E943913DD27CC5D04
:10984000D84F8881F801128218828330F1F048F4F1
:10985000813059F0823081F0DF91CF911F910F91CB
:1098600008958430B9F08530B9F78091AC0D9091AE
:10987000AD0D009789F306C08091AE0D9091AF0DAC
:10988000009799F30E948E22E7CF8091B00D9091BE
:10989000B10DF6CF8091B20D9091B30D009791F775
:1098A0002091AC0D3091AD0D8091AE0D9091AF0D2A
:1098B00021153105F1F2009729F7C901E3CF809115
:1098C000770208950895FC019B0180917713909190
:1098D00078138617970740F0672B29F48091E800EA
:1098E0008E778093E800C90140E0009741F4411170
:1098F00006C08091E80082FF2FC080E0089520918B
:10990000E10B2115A9F12530A9F12091E80023FDF3
:109910002DC02091E80022FDECCF2091E80020FF2F
:10992000E4CF2091F2003091F300009719F0283035
:10993000310558F041E02830310509F040E0209130
:10994000E8002E772093E800D0CF41914093F100BA
:1099500001972F5F3F4FE9CF8091E10B811541F0D7
:10996000853041F08091E80083FFC3CF81E0089506
:1099700082E0089583E008958091711387FF13C0FA
:109980008091E80082FF06C08091E8008B77809389
:10999000E80008958091E10B8111F2CF0895809144
:1099A000E10B8115D9F38091E80080FFF8CF809119
:1099B000E8008E77ECCF982F9093E900891771F02B
:1099C0007091EC002091ED005091F00021FD09C054
:1099D0009F5F973089F78093E9000895762F242FB1
:1099E00050E03091EB003E7F3093EB003091ED0082
:1099F0003D7F3093ED003091EB0031603093EB0010
:109A00007093EC002093ED005093F0002091EE0055
:109A100027FDDECF089590917802913021F4909146
:109A2000621397FD0CC0E8E9F5E09191891302C03B
:109A3000DF011E9255E0EE39F507B9F70895E82FDA
:109A4000E695E695E695803FC8F7F0E0E256FA4FD6
:109A5000877021E030E0A90102C0440F551F8A95AC
:109A6000E2F7CA01809592818923828308951F922B
:109A70001FB61F9211248F939F93AF93BF93809132
:109A8000811390918213A0918313B0918413419616
:109A9000A11DB11D8093811390938213A093831312
:109AA000B0938413BF91AF919F918F911F901FBE70
:109AB0001F9018952FB7F89480918113909182137D
:109AC000A0918313B09184132FBF0895CF93DF9398
:109AD000EC01F0DF8C1B9D0BDF91CF9108952FB728
:109AE000F894609181137091821380918313909107
:109AF00084132FBF089578941F921FB61F921124CC
:109B00008F939F93AF93BF93809181139091821312
:109B1000A0918313B09184130196A11DB11D809370
:109B2000811390938213A0938313B0938413BF91F6
:109B3000AF919F918F911F901FBE1F90189581E04C
:109B40008093E00080E28093D8001092C9008FE1FA
:109B50009EE40197F1F700C0000087E090EBDC0184
:109B60008093851390938613A0938713B0938813E3
:109B700088E19CE00FB6F894A895809360000FBE32
:109B800090936000FFCF2091E4003091E50095E6CE
:109B9000A9012091EC00822F817020FF06C08091E6
:109BA000E80080FF06C080E008952091E80022FDD3
:109BB0001AC08091E10B811589F0853089F0809180
:109BC000EB0085FD0FC02091E4003091E5004217C5
:109BD0005307F9F29A95E1F684E0089582E008953A
:109BE00083E0089581E00895A0E0B0E0EAEFFDE4AD
:109BF0000C941D5FC8EDD0E088818F7E8883E7EDEF
:109C0000F0E080818160808381E08093701388819F
:109C10008C7F888302EE10E0D8011C921092DA004B
:109C200081EEC82ED12CD6011C9288818F77888333
:109C300088818068888388818F7D8883808180681F
:109C4000808319BC1092E10B10926F1310926E1367
:109C500010926D1390EEE92EF12CF70180818B7F2D
:109C6000808388818160888342E060E080E0A3DEB9
:109C7000D6018C918E7F8C93F801808181608083E6
:109C8000808188608083D7018C918E7F8C938881BE
:109C900080618883CDB7DEB7E8E00C94395FE8EDEA
:109CA000F0E080818C7F80831092E2001092DA00D5
:109CB0001092E100A0EEB0E08C9181608C938081E5
:109CC0008F77808319BCA7EDB0E08C918E7F8C9349
:109CD00080818F7E80831092701308951F920F925F
:109CE0000FB60F9211240BB60F922F933F934F9301
:109CF0005F936F937F938F939F93AF93BF93EF93F4
:109D0000FF938091E10082FF09C08091E20082FF11
:109D100005C08091E1008B7F8093E1008091DA00A3
:109D200080FF22C08091D80080FF1EC08091DA00A1
:109D30008E7F8093DA008091D90080FFAEC084E1ED
:109D400089BD86E189BD09B400FEFDCF81E0809325
:109D5000E10B80917013811107C0A1DF45DF809175
:109D6000E20084608093E2008091E10080FF1AC0ED
:109D70008091E20080FF16C08091E2008E7F809388
:109D8000E2008091E20080618093E2008091D8003F
:109D900080628093D80019BC85E08093E10B83E05A
:109DA000809379028091E10084FF35C08091E200C8
:109DB00084FF31C084E189BD86E189BD09B400FE1C
:109DC000FDCF8091D8008F7D8093D8008091E100F5
:109DD0008F7E8093E1008091E2008F7E8093E2008D
:109DE0008091E20081608093E20080916F13811581
:109DF00009F459C084E08093E10B0E94D81A0E94B4
:109E0000BE1810924A0A8091E10B843009F053C0C9
:109E100082E0809379028091E10083FF2BC08091E2
:109E2000E20083FF27C08091E100877F8093E100FB
:109E300082E08093E10B10926F138091E1008E7F9E
:109E40008093E1008091E2008E7F8093E200809118
:109E5000E20080618093E20042E060E080E0ABDD00
:109E60008091F00088608093F00081E08093790217
:109E700080937802FF91EF91BF91AF919F918F9165
:109E80007F916F915F914F913F912F910F900BBEFA
:109E90000F900FBE0F901F90189519BC1092E10BF8
:109EA0001092701361CF8091E30087FF02C083E0BE
:109EB000A2CF81E0A0CF81E0ACCFAAE2B0E0E3E6A0
:109EC000FFE40C94225F81E793E1FC01019620916D
:109ED000F100208323E189379207B9F7809172134B
:109EE000893009F458C0C8F4823009F4B3C0833013
:109EF00009F483C0813089F18091E80083FFE7C0D5
:109F000080917113909172139A3008F0E0C0E92F9C
:109F1000F0E0E455FE490C945D5F8A3009F48AC094
:109F20008B3051F780917113813231F78091751325
:109F300090917613892B01F78091E800877F8093B9
:109F4000E8001ADD81E090917313911101C080E067
:109F5000809378020E94D81ACFCF80917113813AF2
:109F600059F68091E800877F8093E800809175130F
:109F700090917613892B59F060E080E090E070E0DA
:109F8000A2DC8091E8008B778093E800B5CF68E091
:109F900089E793E1F4CF80917113813209F0ACCF5E
:109FA00080917513909176138D7F892B09F0A4CF42
:109FB0008091E800877F8093E8008091E80082FF2D
:109FC00017C08091F2009091F300029731F48091D4
:109FD000F100813011F0863021F48091F1008093FE
:109FE00077028091E8008B778093E800C5DC84CF0E
:109FF0008091E10B8111E1CF7FCF80917113813A84
:10A0000009F07ACF8091751390917613892B09F01E
:10A0100073CF8091E800877F8093E8008091E8000B
:10A0200080FFFCCF809178028093F1008091E8005E
:10A030008E77DACF80917113813209F05DCF8091F4
:10A04000E800877F8093E80097DC80917413809309
:10A05000760252CF80917113813A09F04DCF8091F1
:10A06000E800877F8093E8008091E80080FFFCCFC4
:10A0700080917602D9CF803889F0823841F580917D
:10A0800075138F70873018F58093E9008091EB008D
:10A0900085FB882780F91092E90006C080916E1335
:10A0A000880F90916D13892B9091E800977F909382
:10A0B000E8008093F1001092F1008091E8008E7723
:10A0C00023C0811116C080917313813009F18091F2
:10A0D000E80083FF0AC08091E800877F8093E80052
:10A0E0008091EB0080628093EB00AA96E3E00C94F1
:10A0F0003E5F823061F780917313811581F0109279
:10A10000E9008091E800877F8093E80035DCDFCFAD
:10A1100081E0933009F080E080936E13F0CF80915E
:10A1200075138F702FEF280F263088F68093E90083
:10A130002091EB0020FFE3CF933031F48091EB00CE
:10A1400080628093EB00DBCF9091EB009061909365
:10A15000EB0021E030E0A90102C0440F551F8A95B1
:10A16000E2F74093EA001092EA008091EB008860E9
:10A17000E8CF8111ACCF109173131F778091E3006A
:10A180008078812B8093E3008091E800877F809323
:10A19000E800F2DB8091E80080FFFCCF8091E300D3
:10A1A00080688093E30083E0111101C082E0809316
:10A1B000E10B8DCF8058823008F089CF80917313E6
:10A1C000909174138C3D53E0950791F583E08A8359
:10A1D0008AE289834FB7F894DE01139620E03EE0CF
:10A1E00051E2E32FF0E050935700849120FF03C029
:10A1F00082958F703F5F8F708A30C0F0895C90E0ED
:10A200008D939D932F5F243161F74FBF8091E800BC
:10A21000877F8093E8006AE270E0CE01019653DB0D
:10A220008091E8008B778093E80051CF805DE7CF85
:10A23000292F33272330310509F44EC078F521301A
:10A24000310509F488C08FEB90E0E3E9F8E02230B3
:10A25000310509F03CCF2091E800277F2093E800EA
:10A2600020917713309178138217930708F49C019B
:10A2700040E02115310509F073C0411171C0809192
:10A28000E80082FDCDCF8091E10B811549F2853048
:10A2900039F28091E80083FFF2CFC2CF809175132D
:10A2A000909176132132310509F446C022323105EE
:10A2B00009F00DCF8330910508F009CFFC01EE0FB6
:10A2C000FF1FE857FA4F0190F081E02D8B579A4F0E
:10A2D000DC018C9190E010C09C013327823021F189
:10A2E0002330310568F4232BB9F4EAEAF9E0E4916C
:10A2F0008E2F90E0EAEAF9E0009709F4E8CEABCFC0
:10A300002330310509F0E3CEE4E6F9E0E4918E2F45
:10A3100090E0E4E6F9E0F0CFEEE9F9E0E4918E2F89
:10A3200090E0EEE9F9E0E8CFE2E8F9E0E4918E2F81
:10A3300090E0E2E8F9E0E0CF8330910508F0C7CE85
:10A34000FC01EE0FFF1FE257FA4F0190F081E02D64
:10A3500089E090E080CF82E190E0E2E5F9E07BCF18
:10A360008091E10B811509F45BCF853009F458CF5A
:10A370008091E80083FD54CF8091E80082FD7FCF7B
:10A380008091E80080FF75CF8091F2009091F300FA
:10A390002115310519F08830910550F041E00897FA
:10A3A00009F040E08091E8008E778093E80061CF6B
:10A3B00044914093F1003196215031090196E8CF44
:10A3C000803809F084CE8091E800877F8093E80090
:10A3D00080916F138093F10070CE811178CE10912F
:10A3E0007313123008F073CE8091E800877F80935A
:10A3F000E80010936F13C0DA111519F184E080930F
:10A40000E10B42E061EC81E0D6DA42E261EC84E00B
:10A41000D2DA42E261EC82E0CEDA42E260EC83E042
:10A42000CADA42E361E885E0C6DA42E360E886E042
:10A43000C2DA8091E10B843051F482E0809379029A
:10A4400046CE8091E30087FDD9CF81E0D8CF81E06F
:10A45000F5CF1F920F920FB60F9211240BB60F92E9
:10A46000EF92FF920F931F932F933F934F935F931E
:10A470006F937F938F939F93AF93BF93CF93EF93FC
:10A48000FF9309EE10E0F8018081C091EC008F701D
:10A49000C795CC27C795C82B108280EFE82EF12CEA
:10A4A000F7018081877F8083789407DDF80110822F
:10A4B000F701808188608083CF70F801C083FF91AD
:10A4C000EF91CF91BF91AF919F918F917F916F91BC
:10A4D0005F914F913F912F911F910F91FF90EF90BE
:10A4E0000F900BBE0F900FBE0F901F901895EF921C
:10A4F000FF920F931F93CF937C018B0144DBC82FF6
:10A50000811116C08091E80085FD0AC08091E800A5
:10A510008E778093E80037DB8115A1F3C82F08C040
:10A52000F70181917F018093F1000150104051F7B4
:10A530008C2FCF911F910F91FF90EF900895282FAE
:10A54000CB01BA013091E10B3430C9F42093E9001A
:10A550002FEF3091E80035FD06C035ED3A95F1F763
:10A5600000002A95B1F72091E80025FF08C040E0DF
:10A5700050E0BDDF8091E8008E778093E800089579
:10A58000792F603229F440E250E0682F82E0D7CF83
:10A590000895CF93DF93D82FC92F48E050E0682F5C
:10A5A000792F81E0CCDF88E0ED2FFC2FA9E7B3E124
:10A5B00001900D928A95E1F7DF91CF910895BC014A
:10A5C00040E250E084E0BBCFBC0143E050E084E0D7
:10A5D000B6CFEF92FF920F931F93CF937C018B0125
:10A5E000D2DAC82F811116C08091E80085FD0AC01B
:10A5F0008091E8008B778093E800C5DA8115A1F39C
:10A60000C82F08C08091F100F70181937F010150AC
:10A61000104051F78C2FCF911F910F91FF90EF9029
:10A620000895E091080CF091090C309739F00284FC
:10A63000F385E02D309711F060E209950895A3E0CD
:10A64000B0E0E5E2F3E50C941D5F7C01162FD42EFB
:10A65000C22E8091700A843069F5E091650AF0910C
:10A66000660A3097B9F1970121503109C90163E0B9
:10A6700070E00E94FF5EB901681B790B19834A8361
:10A68000CB824E2D461B9E012F5F3F4F8BE49AE0FD
:10A690000995E091690AF0916A0A309739F00C2D1A
:10A6A0002D2D412FB7018BE49AE009952396E8E020
:10A6B0000C94395F82E0E816F10409F454C083E099
:10A6C000E816F104A9F081E0E816F10409F47AC073
:10A6D000E12CF12CE091670AF091680A3097C9F2F9
:10A6E0000C2D2D2D412FB7018BE49AE00995D1CF88
:10A6F000862F807F803B19F188F4803929F1803AD8
:10A7000041F1E091510AF091520A803819F73097DF
:10A7100009F32C2D4D2D612F6F700DC0803EF1F08F
:10A72000803FC1F6623FB1F6E091570AF091580AB6
:10A7300062EF309779F28BE49AE00995AACFE09125
:10A740004D0AF0914E0AE3CFE0914F0AF091500A82
:10A75000DECFE091530AF091540AD9CFE091550A27
:10A76000F091560AD4CF862F807F803D81F0803FC4
:10A7700099F0E091590AF0915A0A803C09F0AACF69
:10A78000309709F4A7CF4D2D612F6F7017C0E0915E
:10A790005B0AF0915C0AF4CFE0915D0AF0915E0AE9
:10A7A000633F39F0613F09F095CFE0915F0AF09186
:10A7B000600A4D2D612F309709F48CCF8BE49AE01D
:10A7C000099567CFE091610AF091620A683F38F419
:10A7D000663F09F07FCFE091630AF091640A3097F9
:10A7E00009F478CF612F8BE49AE0099552CFAF92AC
:10A7F000BF92DF92EF92FF920F931F93CF93DF935D
:10A800005C01809164020E942518C82F192F609165
:10A81000D30B66958091460A9091470A0E942217B1
:10A82000D82ED0E0CE01880F991F9C012A5A3B4FA9
:10A8300079011C1709F070F481E0113308F080E011
:10A84000DF91CF911F910F91FF90EF90DF90BF901C
:10A85000AF900895FE01E851FB4F80819091650211
:10A8600089238115B9F0F70121A92052330B40A9A2
:10A870004057550B6091D00B7091D10B8091D20B4A
:10A880000D2DF50109950E947D15472F282FCE012A
:10A890000E942218F2E0EF0EF11C2196CACFA0E030
:10A8A000B0E0E5E5F4E50C94175F3C0180916402AB
:10A8B0000E942518C82F192F6091D30B669580919F
:10A8C000460A9091470A0E942217F82ED0E0CE0146
:10A8D000880F991F9C012A5A3B4F69011C1709F0E8
:10A8E00048F481E0113308F080E0CDB7DEB7EEE048
:10A8F0000C94335FFE01E851FB4F8081909165021B
:10A900008923811571F1F60180A9282F2057330B77
:10A91000590181A9E82FE052FF0B4F01AA9C900139
:10A92000AB9C300D300D1124EE9FC001EF9F900DB8
:10A93000900D1124820F931F0E944117082F6091E0
:10A94000D00B7091D10B8091D20BEF2C9401A5010B
:10A95000F30109950E947D15472F282FCE010E94F3
:10A960002218F2E0CF0ED11C2196B8CFA4E0B0E0BF
:10A97000ECEBF4E50C941D5F6C01809164020E9485
:10A9800025188B83F92E6091D30B6695669580917F
:10A99000460A9091470A0E942217182F80E4810FDF
:10A9A0000E94B71780588983812F0E94B71780585B
:10A9B0008A839B81892F90E09C838B839B819F1549
:10A9C00048F081E0E1E3FE1608F080E02496E8E03C
:10A9D0000C94395FEB81FC81E851FB4F80819091B1
:10A9E000650289238115A1F06091D00B7091D10B84
:10A9F0008091D20BE12E0B812A814981F6010995C4
:10AA00000E947D15472F282F8B819C810E94221840
:10AA10008B819C810196D0CFA0E0B0E0E2E1F5E52A
:10AA20000C941E5FC82FD0E0FE01E851FB4F8081DF
:10AA3000909165028923811541F1D090D10B00914D
:10AA4000D20B1091D00BE12EF12C83E00E94AE17B7
:10AA5000482FC7018C549F4F68E671E00E944A5FFF
:10AA60008E199F0997FD03969595879595958795DE
:10AA7000612F489F600D11247D2D802F0E947D1530
:10AA8000472F282FCE010E942218CDB7DEB7E7E06E
:10AA90000C943A5F1F93CF93DF93C82FD0E0FE0151
:10AAA000E851FB4F8081909165028923811591F0D7
:10AAB0000E949917182F80E80E94AE177FE7780F41
:10AAC000612F8091D20B0E947D15472F282FCE0138
:10AAD0000E942218DF91CF911F910895EF92FF926B
:10AAE0000F931F93CF93DF937C01809164020E94A8
:10AAF0002518C82F192F6091D30B6695669521E014
:10AB0000620F08F46FEF8091460A9091470A0E9405
:10AB10002217082FD0E0C11748F081E0113308F068
:10AB200080E0CDB7DEB7E6E00C943B5FFE01E85174
:10AB3000FB4F8081909165028923811589F0609196
:10AB4000D00B7091D10B8091D20B202F4C2FF7019D
:10AB500009950E947D15472F282FCE010E942218AB
:10AB60002196D9CFA0E0B0E0E8EBF5E50C941C5FAE
:10AB70008C01809164020E942518C82FD92E209143
:10AB8000D30B31E0230F08F42FEF30E040E050E02A
:10AB90006FEF7FEF80E090E00E946A607901D0E083
:10ABA000C22EBF2C2C2FCD1550F081E0F1E3DF1623
:10ABB00008F080E0CDB7DEB7E9E00C94385FFE0125
:10ABC000E851FB4F8081909165028923811511F135
:10ABD00040911C0A4150042E000C550B47FF1CC02D
:10ABE0008C2D9B2D6091D30B21E0620F08F46FEF49
:10ABF0000E942217AC016091D00B7091D10B809113
:10AC0000D20BF80109950E947D15472F282FCE0100
:10AC10000E9422182196C6CFFA01E45EF54F818981
:10AC200082130AC0FA01EE0FFF1FE45EF54F818D1B
:10AC3000928D8E159F05B0F241505109CFCFA8E0FB
:10AC4000B0E0E5E2F6E50C94135F382E6A837B836F
:10AC5000809164020E942518192F20911C0A2E83CE
:10AC6000E82FF0E0F887EF83CF01880F991F9C0150
:10AC70002A5A3B4F6901432C512C3FEF431A530A88
:10AC80008F81811740F081E0113308F080E0289631
:10AC9000E2E10C942F5FEF81F885E851FB4F808152
:10ACA0009091650289238115F1F08091D00B8C83FE
:10ACB0009091D10B9D83F201E45EF54F3F01232C6F
:10ACC0001982FE812F16C8F06091D20B89810E94F3
:10ACD00004166C817D810E947D15472F282F8F815E
:10ACE00098850E9422182F8138852F5F3F4F388723
:10ACF0002F8332E0C30ED11CC3CFF30181913F01FA
:10AD0000F601A0A8A81ABB0881A8F3018781881AB8
:10AD10009908AA9C9001AB9C300D300D1124889CA1
:10AD2000C001899C900D900D1124820F931F0E94E9
:10AD30004117082F6091D30B21E0620F08F46FEFE9
:10AD4000F301EE0FFF1FEC51FA40858996890E94AE
:10AD500022177C019401A5016C817D818981EA81A2
:10AD6000FB8109956C837D8389832394AACFA0E01E
:10AD7000B0E0EDEBF6E50C941C5FEC0188818115E9
:10AD8000F1F0813009F042C08981813029F48A8153
:10AD900023960E94CD1AF2CF823029F48A8123961D
:10ADA0000E94A619EBCF833029F48A8123960E9452
:10ADB0005B1AE4CF843041F022968111DFCFCDB70A
:10ADC000DEB7E9E00C94385F8A81239620E030E01A
:10ADD0009AE0682F6053770BAB016A30710560F021
:10ADE0002115310551F3EFE9FFE03197F1F700C08C
:10ADF000000021503109F4CF929FB001939F700D54
:10AE000011249A01260F371F8991E3CFE82FF0E034
:10AE1000ED5EF74FB490282F26952695269530E0C5
:10AE2000F901ED5FF74FE4908770F12C082E02C016
:10AE3000F594E7940A94E2F7E0FAEE24FF24E0F8B0
:10AE4000F901ED50F84FC490D12C082E02C0D594D2
:10AE5000C7940A94E2F7C0FACC24DD24C0F8F901C3
:10AE6000ED51F84F049110E002C0159507958A95B1
:10AE7000E2F701701127E114F10419F081EE0E944C
:10AE8000A619C114D10419F086EE0E94A61960E03B
:10AE900070E08B2D0E94B71AC114D10419F086EE10
:10AEA0000E945B1AE114F10419F081EE0E945B1A12
:10AEB0000115110519F08CE20E94CD1A21965ECF82
:10AEC000CF92DF92EF92FF92CF93DF93EC017B0161
:10AED0008091B60D80FD09C00E943614DF91CF919C
:10AEE000FF90EF90DF90CF9008958091E608811158
:10AEF00002C00E945F148091A30881110E94361441
:10AF000081E08093A40810928E08D0938D08C0939E
:10AF10008C08E0929008F092910810928F0810929D
:10AF20009308109292086C817D818E819F8117D742
:10AF30009B01A3E5B7E00E94B86020EFC22ED12CA0
:10AF4000E12CF12CA70196010E949660688179811D
:10AF50008A819B81A9010E94521F0E945A4D9093A1
:10AF6000F9088093F808E0918C08F0918D088091A1
:10AF700092089091930833E0880F991F3A95E1F772
:10AF8000E80FF91F6481758186819781E8D69B015E
:10AF9000A3E5B7E00E94B860A70196010E94966001
:10AFA0003093A2082093A10899CF1F93CF93DF93EA
:10AFB000182FA091B80FB091B90F109709F44AC09B
:10AFC0001092BB0F1092BA0F1092D60D1092D50DA1
:10AFD0001696CD91DC911797CE019A9581159F41D8
:10AFE00008F4D07ED1E0C11101C0D0E01996ED91F6
:10AFF000FC911A97309731F01B966D917C9180E00F
:10B000000995D823D11539F08CEF8C0F813A30F5A2
:10B010008C2F0E940B4D1115A9F0E091B80FF09103
:10B02000B90F808584FD0EC08091B70F811551F056
:10B03000808191819C01215031092F333E4710F4CA
:10B040000E9469180E942F191092B90F1092B80F20
:10B050001092B70FDF91CF911F9108950E942F1981
:10B060008C2F0E945B1AD7CF611529F02091DD113A
:10B0700022602093DD119C0130522115304308F4E9
:10B0800099270C94461AFF920F931F93CF93DF9347
:10B09000EC018B01F42E80913F0382FF69C0209167
:10B0A000C8113091C9112C173D0719F0209709F0EC
:10B0B0005FC090913F039B7F90933F0361E091FDC0
:10B0C00010C08091C6119091C711A801481B590B5F
:10B0D00061E080915C0290915D024817590708F485
:10B0E00060E080913F0360FB81F980933F03C901D9
:10B0F0000E942E188091DA1181FF08C080913F03D1
:10B10000806180933F0382E00E94B1138091DA1145
:10B1100085FF08C080913F03806280933F0380E2F7
:10B120000E94B11360913F03669561708091C811D0
:10B130009091C91199DFF11431F08091551385FF79
:10B1400002C086FF29C080915813909159130E9424
:10B1500039138091C8119091C9119C013052211569
:10B16000304308F499270E94A21A0E94611C10C063
:10B17000CE0190528115904398F4CE0199270E94F8
:10B18000A21A8091C8119091C911C817D90769F303
:10B190001093C7110093C611CDB7DEB7E5E06CC6BA
:10B1A000CE01EDCFAAE0B0E0E7EDF8E54CC69C019A
:10B1B00097558115914068F4BE016F5F7F4F822FD4
:10B1C0000E945418892B29F489859A852A96E2E0F1
:10B1D00056C68091521390915313F8CFA0E0B0E07F
:10B1E000E3EFF8E52BC6162FD72FC42FD22E8115EB
:10B1F000A1F04093D3110E945A4D90936C13809309
:10B200006B13C77081E001C0880FCA95EAF70E94EE
:10B210008319CDB7DEB7E7E02DC69091D31149135E
:10B2200037C0E0906B13F0906C130E945A4D9C0154
:10B230002E193F097901812F9D2FB4DFE816F906F9
:10B2400038F5D0E2DD0DCD15A1F0C77011E0812FEA
:10B2500001C0880FCA95EAF70E949219D83048F4C5
:10B260008D2D877001C0110F8A95EAF7812F0E94FA
:10B270008319802F0E94CD1AD83058F62D2D2770B3
:10B2800081E001C0880F2A95EAF70E949219C1CF88
:10B29000C77081E001C0880FCA95EAF7F6CFA8E031
:10B2A000B0E0E4E5F9E5C3C5FE01319688E0DF01D1
:10B2B0001D928A95E9F796E4A92E94E0B92E8F01A4
:10B2C0003F01EE24E394F12C36E5C32E34E0D32E77
:10B2D000F50181915F018F3F09F444C0F894E82F94
:10B2E000E295EF70F0E021A18F70A70102C0440F3A
:10B2F000551F8A95E2F7CA01922F982B91A392A12C
:10B300008095892382A3789400C0EAE4F4E021E0E8
:10B3100030E0812C912C41914F3F79F0A42FA295E0
:10B32000AF70A05EB0E08C9190E04F7002C0959538
:10B3300087954A95E2F780FF39C080E090E0882A3F
:10B34000992A220F331FCE16DF0629F7F5018291C5
:10B350008F3F11F00E941D1450EA5A95F1F7D80161
:10B360008D929C920E5F1F4FBAE4AB16B4E0BB0601
:10B3700009F0AECF48E050E0B30187EE98E01BD66D
:10B38000892BB1F088E0F301A7EEB8E001900D92AF
:10B390008A95E1F781E080936A130E945A4D909359
:10B3A0006913809368132896EEE05DC5C901C7CF85
:10B3B00080916A138115B9F3009168131091691394
:10B3C0000E945A4D801B910B059768F348E050E0AE
:10B3D00067EE78E087ED9BE0EED5892B49F088E0B9
:10B3E000E7EEF8E0A7EDBBE001900D928A95E1F75A
:10B3F00010926A13D8CFE0918B0C90918A0C29E0BF
:10B40000E91302C080E00895AE2FB0E02E9FF00156
:10B410001124ED5DF34F3181361306C030813813AE
:10B4200003C03581341304C0FD013196E770E8CFC5
:10B4300081E00895CF93DF930E94D81A0E9465158A
:10B440000E94AC180E945A4DEC0163E070E081EA62
:10B4500093E036DD0E945A4D8C1B9D0B8A3F91056F
:10B4600028F00E943614DF91CF9108958FE99FE074
:10B470000197F1F700C00000EDCF1F93CF93DF934A
:10B48000182FD92F611599F0411589F00E94D41316
:10B49000C82F682F812F9D2F0E944713612F7D2F6A
:10B4A0008C2F0E94B913DF91CF911F9108950E94B4
:10B4B0007D13C82FF3CFFF920F931F93CF93DF938A
:10B4C000182FEB011092BC0084EA8093BC000E940C
:10B4D0005A4D082FF92E8091BC0087FF28C080911B
:10B4E000B900887F883029F08091B900887F803149
:10B4F00099F51093BB0084E88093BC000E945A4DDC
:10B50000182F092F8091BC0087FF1EC02091B90021
:10B51000287F80E090E0283199F081E090E02034AD
:10B5200011F480E090E091958195910909C0802FF8
:10B530009F2D0E94664DC817D90768F68EEF9FEFC2
:10B54000CDB7DEB7E5E098C4812F902F0E94664DFD
:10B55000C817D907B8F6F2CF8FEF9FEFF1CF10924F
:10B56000B9008CE08093B80008950F931F93CF9398
:10B57000DF93EB018093BB0084E88093BC000E94C2
:10B580005A4D182F092F8091BC0087FF11C02091C0
:10B59000B900287F81E090E0283211F480E090E04B
:10B5A000919581959109DF91CF911F910F91089508
:10B5B000CF3FDC0741F3812F902F0E94664DC817C3
:10B5C000D90708F78EEF9FEFEECFA0E0B0E0EAEEEC
:10B5D000FAE52DC4682E962E5A01690178010E9461
:10B5E0005A4D782E892E0431110518F10F3F10079E
:10B5F00019F1C80164E170E002D4162F072F612F02
:10B60000702F862D58DFEC01892BC1F0FFEFEF166C
:10B61000FF06A9F3872D982D0E94664DE816F906BE
:10B6200070F784E98093BC00CE01CDB7DEB7EEE0C1
:10B630001AC411E000E0E3CF15E0FCCFB701892D7B
:10B6400094DFEC018501CA0CDB1C0C151D0549F3C8
:10B65000209739F7B701F80181918F0186DFEC015E
:10B66000F4CF5ED018F011F062D038F456C089C023
:10B67000E92F64D0B0F35523C9F3E7FB62177307D2
:10B6800084079507A8F199F3E92FFF2788232AF06B
:10B690003197660F771F881FDAF7952F55274423B8
:10B6A00032F091505040220F331F441FD2F7BB2776
:10B6B000E91BF50B621B730B840BB109C1F222F479
:10B6C000620F731F841FB11D31972AF0660F771F19
:10B6D000881FBB1FEFCF915050405AF041F0882394
:10B6E00032F0660F771F881F91505040C1F7939535
:10B6F00006C08695779567959F5FD9F7F8CF9F3FEE
:10B7000031F0915020F4879577956795B795880F1C
:10B71000911D9695879597F908959FEF80EC089570
:10B7200000240A9416161706180609060895002420
:10B730000A941216130614060506089557FD90582C
:10B74000440F551F59F05F3F71F04795880F97FBE5
:10B75000991F61F09F3F79F087950895121613069F
:10B760001406551FF2CF4695F1DF08C016161706CE
:10B770001806991FF1CF8695710561050894089503
:10B78000E894BB2766277727CB0197F90895FA013C
:10B79000EE0FFF1F30962105310599F161157105F6
:10B7A00061F48038BFE39B0749F1689490388105C4
:10B7B00061F08038BFEF9B0741F0992342F5FF3FCE
:10B7C000E1053105210511F1E8940894E795D901C7
:10B7D000AA2329F4AB2FBE2FF85FD0F310C0FF5F70
:10B7E00070F4A695E0F7F73950F019F0FF3A38F405
:10B7F0009F779F930CD00F9007FC905808953EF0D0
:10B800008CCF60E070E080E89FE308954FE79F777A
:10B810005F934F933F932F93A6D02F913F914F91DA
:10B820005F9116D105C019F40EF02FC0A9CF75CFC6
:10B830008DDFC8F39638C0F707F80F92E8942BE332
:10B840003AEA48EB5FE712D10F920F920F924DB791
:10B850005EB70F92CAD0E2E9F1ECB0E01CD04F9194
:10B860005F91EF91FF91E595EE1FFF1F49F0FE57A5
:10B87000E0684427EE0F441FFA95E1F74195550B18
:10B8800039D00F9007FE2DC0089597F99F6780E883
:10B8900070E060E00895DF93CF931F930F93FF92C2
:10B8A000EF92DF92BBBF7B018C01689405C0DA2E5A
:10B8B000EF01DAD0FE01E894A791279137914791E3
:10B8C0005791AEF3EF0139D1FE019701A801DA9447
:10B8D00079F7DF90EF90FF900F911F91CF91DF915B
:10B8E00008959B01AC0160E070E080E89FE378C1BF
:10B8F000CCCF05CF2BDFE8F39923D9F3940F511D5B
:10B90000BBF39150504094F059F0882332F0660F09
:10B91000771F881F91505040C1F79E3F510544F753
:10B92000880F911D9695879597F908955F3FACF024
:10B93000983E9CF0BB27869577956795B79508F458
:10B94000B1609395C1F7BB0F58F711F460FFE8CFD2
:10B950006F5F7F4F8F4F9F4FE3CF13CF0EF0CFCE50
:10B96000DCCE689492CFF2DEC8F39923D1F3C6F30C
:10B97000DF93CF931F930F93FF92C92FDD27882367
:10B980002AF02197660F771F881FDAF720E030E052
:10B9900040E85FEB9FE3883920F0803E38F0219645
:10B9A0008F77BAD0EAEBF1ECB0E004C0B5D0E7EEA7
:10B9B000F1ECB0E070DF8B01BE01EC01FB2E6F57A4
:10B9C00071097595771F880B990B74D128E132E7BF
:10B9D00041E35FE349D0AF2D9801AE01FF900F9195
:10B9E0001F91CF91DF91A9D0A0C1FA01DC01AA0F6C
:10B9F000BB1F9B01AC01BF5728F4222733274427E4
:10BA000050781FC0B75188F4AB2F00244695379566
:10BA10002795011CA395D2F3002069F0220F331F54
:10BA2000441FB395DAF30DD076C061307105A0E8FC
:10BA30008A07B94630F49B01AC016627772788272F
:10BA40009078309621F02083318342835383089588
:10BA50000BD06BC165DE28F06ADE18F0952309F083
:10BA600014CF5BCE11248DCE69DEA0F3959FD1F368
:10BA7000950F50E0551F629FF001729FBB27F00D9C
:10BA8000B11D639FAA27F00DB11DAA1F649F6627F1
:10BA9000B00DA11D661F829F2227B00DA11D621F40
:10BAA000739FB00DA11D621F839FA00D611D221FFA
:10BAB000749F3327A00D611D231F849F600D211DDE
:10BAC000822F762F6A2F11249F5750408AF0E1F081
:10BAD00088234AF0EE0FFF1FBB1F661F771F881FCA
:10BAE00091505040A9F79E3F510570F0CECE49CEFF
:10BAF0005F3FECF3983EDCF3869577956795B795B5
:10BB0000F795E7959F5FC1F7FE2B880F911D9695DE
:10BB1000879597F908955058BB27AA270ED005C1DD
:10BB2000FFDD30F004DE20F031F49F3F11F41EF40D
:10BB3000F4CD0EF4E095E7FBA8CEE92FFFDD80F30E
:10BB4000BA17620773078407950718F071F49EF51A
:10BB500017CE0EF4E0950B2EBA2FA02D0B01B901D4
:10BB600090010C01CA01A0011124FF27591B99F073
:10BB7000593F50F4503E68F11A16F040A22F232F7F
:10BB8000342F4427585FF3CF469537952795A795CF
:10BB9000F0405395C9F77EF41F16BA0B620B730B76
:10BBA000840BBAF09150A1F0FF0FBB1F661F771FE7
:10BBB000881FC2F70EC0BA0F621F731F841F48F49C
:10BBC000879577956795B795F7959E3F08F0B3CF22
:10BBD0009395880F08F09927EE0F9795879508950C
:10BBE0000CD0A3C0A4DD40F09BDD30F021F45F3F1A
:10BBF00019F04BCE5111C5CD90CDA0DD98F399230E
:10BC0000C9F35523B1F3951B550BBB27AA27621720
:10BC10007307840738F09F5F5F4F220F331F441F65
:10BC2000AA1FA9F333D00E2E3AF0E0E830D091509D
:10BC30005040E695001CCAF729D0FE2F27D0660F8A
:10BC4000771F881FBB1F261737074807AB07B0E8C9
:10BC500009F0BB0B802DBF01FF2793585F4F2AF0DF
:10BC60009E3F510568F011CE8CCD5F3FECF3983EBE
:10BC7000DCF3869577956795B795F7959F5FC9F73C
:10BC8000880F911D9695879597F90895E1E0660FC5
:10BC9000771F881FBB1F621773078407BA0720F03E
:10BCA000621B730B840BBA0BEE1F88F7E0950895A7
:10BCB000E89409C097FB3EF4909580957095619546
:10BCC0007F4F8F4F9F4F9923A9F0F92F96E9BB27FC
:10BCD0009395F695879577956795B795F111F8CF78
:10BCE000FAF4BB0F11F460FF1BC06F5F7F4F8F4FE3
:10BCF0009F4F16C0882311F096E911C0772321F0D9
:10BD00009EE8872F762F05C0662371F096E8862F70
:10BD100070E060E02AF09A95660F771F881FDAF7C7
:10BD2000880F9695879597F90895092E0394000C2E
:10BD300011F4882352F0BB0F40F4BF2B11F460FFC5
:10BD400004C06F5F7F4F8F4F9F4F089534D008F42A
:10BD500081E0089504D06894B11113CD0895F6DC04
:10BD600088F09F5790F0B92F9927B751A0F0D1F0E4
:10BD7000660F771F881F991F1AF0BA95C9F712C06E
:10BD8000B13081F0FDDCB1E00895FACC672F782F57
:10BD90008827B85F39F0B93FCCF3869577956795DA
:10BDA000B395D9F73EF490958095709561957F4F46
:10BDB0008F4F9F4F0895990F0008550FAA0BE0E889
:10BDC000FEEF16161706E807F907C0F0121613065D
:10BDD000E407F50798F0621B730B840B950B39F49D
:10BDE0000A2661F0232B242B252B21F408950A2603
:10BDF00009F4A140A6958FEF811D811D0895AA1B0E
:10BE0000BB1B51E107C0AA1FBB1FA617B70710F045
:10BE1000A61BB70B881F991F5A95A9F78095909577
:10BE2000BC01CD0108952F923F924F925F926F9285
:10BE30007F928F929F92AF92BF92CF92DF92EF92BA
:10BE4000FF920F931F93CF93DF93CDB7DEB7CA1B3B
:10BE5000DB0B0FB6F894DEBF0FBECDBF09942A8866
:10BE6000398848885F846E847D848C849B84AA840E
:10BE7000B984C884DF80EE80FD800C811B81AA819B
:10BE8000B981CE0FD11D0FB6F894DEBF0FBECDBF66
:10BE9000ED01089597FB072E16F4009406D077FD68
:10BEA00008D0ADDF07FC05D03EF4909581959F4FFB
:10BEB0000895709561957F4F0895EE0FFF1F002440
:10BEC000001C0BBE0790F691E02D0994082E81709E
:10BED00006940694811D0694811D0694811D069486
:10BEE000811D0694811D0694801D0895692796275B
:10BEF000692778278727782708958F929F92AF9296
:10BF0000BF92CF92DF92EF92FF92CF93DF93EC013B
:10BF1000688179818A819B8161157105810591050F
:10BF200021F464E279ED8BE597E02DE133EF41E018
:10BF300050E0D0D049015A019B01AC01A7EAB1E41D
:10BF4000E5D06B017C01ACEEB4EFA5019401EAD021
:10BF5000DC01CB018C0D9D1DAE1DBF1DB7FF03C0C5
:10BF60000197A109B04888839983AA83BB839F77EF
:10BF7000DF91CF91FF90EF90DF90CF90BF90AF9087
:10BF80009F908F900895B9CF80E091E0B6CFA0E068
:10BF9000B0E08093000190930101A0930201B0935F
:10BFA00003010895FB01DC0102C005900D92415090
:10BFB0005040D8F70895FB01DC0104C08D91019039
:10BFC000801921F441505040C8F7881B990B0895FF
:10BFD000FB01DC0102C001900D9241505040D8F7A6
:10BFE00008956817790768F4FB01DC01E40FF51F79
:10BFF000A40FB51F02C002900E9241505040D8F7D6
:10C000000895E6CFDC0101C06D9341505040E0F748
:10C010000895DC01CB01FC01F999FECF06C0F2BD09
:10C02000E1BDF89A319600B40D9241505040B8F7F6
:10C030000895F999FECF92BD81BDF89A992780B5F0
:10C040000895A8E1B0E042E050E0E5CFDC01A40FA4
:10C05000B51F4150504040F0CB01840F951F2E91E9
:10C0600005D041505040D8F70895262FF999FECFBA
:10C0700092BD81BDF89A019700B4021639F01FBA3B
:10C0800020BD0FB6F894FA9AF99A0FBE0895039658
:10C09000272FECDFEADF252FE9DF242FE7CF0196FA
:10C0A000272FE4DFE2CFDC01CB0102C02D9105D0C8
:10C0B00041505040D8F70895262FF999FECF1FBA66
:10C0C00092BD81BD20BD0FB6F894FA9AF99A0FBEC1
:10C0D00001960895052E97FB16F400940FD057FD96
:10C0E00005D024D007FC02D046F408C050954095F6
:10C0F000309521953F4F4F4F5F4F08959095809514
:10C10000709561957F4F8F4F9F4F089531D0A59FB8
:10C11000900DB49F900DA49F800D911D1124089542
:10C12000B7FFF4CFF3DF821B930B0895A1E21A2E21
:10C13000AA1BBB1BFD010DC0AA1FBB1FEE1FFF1FCB
:10C14000A217B307E407F50720F0A21BB30BE40B1B
:10C15000F50B661F771F881F991F1A9469F7609562
:10C160007095809590959B01AC01BD01CF0108951C
:10C17000A29FB001B39FC001A39F700D811D112428
:10C18000911DB29F700D811D1124911D0895F89489
:10C19000FFCF07634236B79BD8A71A39685618AE47
:10C1A000BAAB558C1D3CB7CC5763BD6DEDFD753EEC
:10C1B000F6177231BF000000803F08000000BE92F9
:10C1C0002449123EABAAAA2ABECDCCCC4C3E0000DC
:10C1D0000080BEABAAAAAA3E00000000BF0000007B
:10C1E000803F0000000000084178D3BB4387D11393
:10C1F0003D190E3CC3BD4282AD2B3E68EC8276BE3B
:10C20000D98FE1A93E4C80EFFFBE01C4FF7F3F0004
:10C2100000000000391D791D7F1D971D741E3B1DF8
:10C22000B91EE21E0D1F962C122D9E2C5A2C5E2C30
:10C23000A22C622CA62CB22C6E2C0B2D722CB62CA0
:10C24000762CBA2CF32C7A2CBE2CFA2C802CC42CF5
:10C25000D82C662CAA2C6A2CAE2C8C2CCE2CE62C3E
:10C26000032D092D542C9A2C192D292C2F2C1B2CE5
:10C27000232C352C3B2C412C5B2D622D2C2D302D6D
:10C28000652D362D6B2D3C2D712D422D772D482D92
:10C290007D2D2C2D302D652D362D6B2D3C2D712DAA
:10C2A000422D772D482D7D2DE84805490B4927461D
:10C2B00027463F4951496349A249A749D349E5491E
:10C2C000FA49FD497D3F883FB33FF33F2D406B4026
:10C2D0008140844087408C408F40944097409A40F2
:10C2E0009D40A040A340A640A940AC40AF40B44010
:10C2F000B740BA40FE404041434146414941A74111
:10C3000073424543D643B244B744BA44C744CB44CE
:10C31000D644D944E444E744F244F5440045034597
:10C320001546194650465F466A4675467846E146C8
:10C3300085471346D24888478B478F47BD47FB4701
:10C34000FE4700483448064A154A2C4A624A834A46
:10C35000A74ABA4ADE4AF84A3B50615067506150DA
:0CC360006750B950DA506750E051ED51C1
:10C36C00010000000000DC44000000410AA7CF449B
:10C37C00000000415CFFB8440000004152D0A444CE
:10C38C00000000411FD59244000000415C978A4494
:10C39C000000004148F176440000004100005C447C
:10C3AC000000004100005C440000004148F176446C
:10C3BC00000000415C978A44000000411FD5924464
:10C3CC000000004152D0A444000000415CFFB8447E
:10C3DC00000000410AA7CF44000000410000DC44EB
:10C3EC00000000410000DC44000000410AA7CF44DB
:10C3FC00000000415CFFB8440000004152D0A4444E
:10C40C00000000411FD59244000000415C978A4413
:10C41C000000004148F176440000004100005C44FB
:10C42C000000004100005C440000004148F17644EB
:10C43C00000000415C978A44000000411FD59244E3
:10C44C000000004152D0A444000000415CFFB844FD
:10C45C00000000410AA7CF44000000410000DC446A
:10C46C0000000041390532010000DC4400000041AD
:10C47C0000005C440000004100005C4400000041EE
:10C48C000000DC44000000415F4CC952DF52624C9A
:10C49C00E452C05252D02445000040415C970A45FA
:10C4AC000000004152D0A444000000410000DC44D4
:10C4BC00000000415C970A450000A041AF0032002B
:10C4CC003200320000FF00FFFF0304854000000132
:10C4DC00064000000100000001000100005C440067
:10C4EC000080415C978A440000804152D0A44400F3
:10C4FC000080410000DC440000804100005C4400EE
:10C50C000080411F1569440000804148F1764400C9
:10C51C0000804100D08244000080415C978A440036
:10C52C00008041A4D024440000804100005C440001
:10C53C000080411FD59244000080415CFFC3440041
:10C54C0000804100000000000000005CFF4344003C
:10C55C000080411FD59244000080410000DC440063
:10C56C0000804152D02445000080410000000000B2
:10C57C0000000000005C440000804148F17644005B
:10C58C000080415C978A44000080411FD592440092
:10C59C0000804152D0A4440000804103640001019A
:10C5AC0000005C440000004100005C4400000041BD
:10C5BC0000005C440000004100005C4400000041AD
:10C5CC0048F176440000C04000005C440000C040CC
:10C5DC0048F176440000C04000005C440000C040BC
:10C5EC0048F176440000C04000005C440000C040AC
:10C5FC0048F176440000C04000005C440000C0409C
:10C60C000152D02445000000410000DC4400000031
:10C61C004152D0A4440000404100FFFF0002040539
:10C62C0007090B0C0E1011131517181A1C1D1F21BE
:10C63C0023242628292B2D2F3032343537393B7BB8
:10C64C00A57F5C134C8D69007476003131295A1B1F
:10C65C00750A030102033149803F5D8B803FF8BFAF
:10C66C00803FCAE1803F73ED803FCAE1803FF8BF55
:10C67C00803F5D8B803F3149803F0000803FF16DF2
:10C68C007F3F75EA7E3F4C827E3F833F7E3F84280E
:10C69C007E3F833F7E3F4C827E3F75EA7E3FF16D4D
:10C6AC007F3F0000803F30C7F0F1C6C3C493949520
:10C6BC00600706C1C09700010203040506070809BC
:10C6CC000A0B0C0D0E0F1011121314151617181946
:10C6DC001A1B1C1D1E1F2021222324252627282936
:10C6EC002B2C2D2E2F300000140028003D00510063
:10C6FC0065007A008E00A200B700CB00DF000015A9
:10C70C00141528153D15511565157A158E15A2159C
:10C71C00B715CB15DF15002A142A282A3D2A512AD1
:10C72C00652A7A2A8E2AA22AB72ACB2ADF2A003F28
:10C73C00143F283F3D3F513F653F6F3F7A3F8E3F4F
:10C74C00A23FB73FCB3FDF3F0104040404040404C1
:10C75C000404040101040404040404040404040196
:10C76C00010404040404040404040401010101018F
:10C77C00010404040101010101E200E900EA00B531
:10C78C0000B600B700CD008301CC008A0192019461
:10C79C00012102230224022502260227022A02B3C7
:10C7AC0000B4006F0070009F01CB019F02A002E259
:10C7BC0000E900EA00B500B600B700CD008301CC5B
:10C7CC00008A0192019401210223022402250226EF
:10C7DC000227022A02B300B4006F0070009F01CB45
:10C7EC00019F02A00244226D9F077D071007A50838
:04C7FC00BE08DE088D
:00000001FF
